:04703E00010002410A
:106AAF00AF50055074D02FF582E4341DF583E5996E
:106ABF00F022D3E5309400E52F94002290000FE0F0
:036ACF006403223B
:030003000258F3AD
:0B58F300C0E0C083C082C0D075D008A8
:1058FE00852E82852D83E493FF201404C4540FFF5C
:10590E00430FF08F80C284D28500C2870000D287F9
:10591E00007580FF7580FEC284C28500C2870000BC
:10592E00D287007580FF30140CC214052EE52E7040
:09593E0006052D8002D214D2A846
:09594700D0D0D082D083D0E03230
:03000B000219696E
:10196900C0E0C0F0C083C082C0D075D008758CD8E3
:10197900758A92D28C1242FA1263F2E531D394003D
:1019890040171531E53164056009E531640F6003DD
:10199900021B7B126CF4021B7B753114E54ED39448
:1019A900004002154EE54FD394004002154FE53A29
:1019B900D394004002153AE54BD394004002154BED
:1019C900154CE54C123A5E1B6D001B42011B1A02B5
:1019D9001AF2031A6F041A56051A3D061A24071A31
:1019E9000B0819F20900001B78D3E52C9400E52BAC
:1019F90094005003021B7BE52C152C704D152B020E
:101A09001B7BD3E5379400E53694005003021B7B1A
:101A1900E537153770021536021B7BD3E54894006C
:101A2900E54794005003021B7BE5481548700215F1
:101A390047021B7BD3E54A9400E549940050030211
:101A49001B7BE54A154A70021549021B7BD3E52A1F
:101A59009400E52994005003021B7BE52A152A709E
:101A6900021529021B7B7884E6FF7003021B7BEFBA
:101A7900B40105900524801BEFB40210126AC1401D
:101A89002FE53015307002152F021B7BEFB4030CC4
:101A9900900526E0F52FA3E0F5308028EFB4041275
:101AA900126AC1400BE53015307002152F021B7BFD
:101AB9008012EF64057003021B7BEFB4060C752FCF
:101AC90002753058788406021B7BEF6407600302B5
:101AD9001B7B126AC1400BE53015307002152F02CD
:101AE9001B7B78847600021B7BD3E5399400E538AB
:101AF90094004008E539153970021538D3E53C944E
:101B090000E53B9400406BE53C153C7002153B80B9
:101B190061D3E5579400E55694004008E5571557F9
:101B290070021556D3E5559400E55494004043E5F9
:101B3900551555700215548039D3E5359400E534AF
:101B490094004008E535153570021534301523D356
:101B5900E5339400E53294004018E53315337012EB
:101B69001532800EE551D39400400415518000755B
:0D1B79004C0AD0D0D082D083D0F0D0E03222
:03001300023B6E3F
:0D3B6E00C0E0C0F0C083C082C0D075D01090
:103B7B00E545C394504003023C3E202403023C3EE7
:103B8B00300C03023C3EE5A0540FF5587D077F0136
:103B9B00124FE55067202364E545700DE558B40CD2
:103BAB0008201105D211023C3E20034A2011471276
:103BBB003C4950047F0180027F0F126FC190000FB0
:103BCB00E0FF64016012EFB40302800C90000FE081
:103BDB00B40209123C4950047F80801290000FE020
:103BEB00B4020E7D037F07124FE540057FA0120044
:103BFB0016754202D20390053CE0F53A7D087F052D
:103C0B00124FE5501A90002BE0B55807202304D231
:103C1B00268020053EE53EAE3D700E053D800A0533
:103C2B003EE53EAE3D7002053D14F5828E83E558B0
:033C3B00F005454C
:103C3E00D0D0D082D083D0F0D0E0327D037F071277
:033C4E004FE5221D
:030023000264CBA9
:1064CB00C0E0C083C082C0D075D018309819C29874
:1064DB00E599B40A08126AAF755000800AE550C3FB
:1064EB0094905003126AAF309902C299D0D0D082E7
:0564FB00D083D0E03267
:03003B000246A0DA
:0D46A000C0E0C0F0C083C082C0D075D0184B
:1046AD00C2CEE546C39410400302474A20250302BB
:1046BD00474A300C0302474AAFA07804EF08800147
:1046CD0023D8FDF55953590F7D077F02124FE55041
:1046DD0035202332E546700CE559B40C0720130440
:1046ED00D213805920041920131690000FE0B40244
:1046FD000F7F0A126FC17F80120016754202D2041D
:10470D0090053CE0F53A7D087F05124FE5501A9073
:10471D00002BE0B55907202304D22880200540E561
:10472D0040AE3F700E053F800A0540E540AE3F703C
:0D473D0002053F14F5828E83E559F0054614
:0B474A00D0D0D082D083D0F0D0E0327D
:104D1E00E4F55AF55B755C1E755DFF855B82855A01
:104D2E0083E0F55E635EFFE55EF0E0655E600312B4
:104D3E007042635EFF855B82855A83E55EF0E065B7
:104D4E005E6003127042055BE55B7002055AE55D1D
:104D5E00155D7002155CD3E55D9400E55C94005022
:104D6E00BA75985A758921758845758DE77587804E
:104D7E00758CD8758AEF75C90275C808753D1E7594
:104D8E003E60753F1E7540B075B701D2A9D2E8D20C
:0F4D9E00AA75C64C75EEFF75FEFFD2AF1267FA0D
:014DAD0022E3
:0270420080FECE
:106A8C00202F0F90053AE0F54EE54ED394004012BE
:106A9C0080F7302F0D90053AE0F54FE54FD3940079
:036AAC0050F9227C
:106A440030310AD215900024E04420800DC2157F15
:106A540008127002900024E054DFF0FD7F247E00D1
:046A64001264952201
:102ECA008F6AE56A640170292030047F01805620E8
:102EDA003003022FC5122FD64003022FC5122FDE50
:102EEA00500C122FC6301503022FC5022FBB022F1A
:102EFA007BE56A640270202030047F02802720303C
:102F0A0003022FC5122FE64003022FC5126ACB70A7
:102F1A0003022FC5022F95E56A64036003022FC5D9
:102F2A002030057F03027002303024122FD6501F42
:102F3A00122FE6501A126ACB6015122FDE500B7F41
:102F4A000B122FEE201574022FBB7F03022FC23003
:102F5A003023122FFC501E7D017F02124FE54015CF
:102F6A007D017F07124FE55008122FC620154C80AD
:102F7A00407F018043303017122FFC40127D017FC1
:102F8A0002124FE55009126ACB60047F0280293091
:102F9A0030297D017F01124FE55020126ACB701B48
:102FAA007D017F07124FE5500D7F09122FEE201584
:102FBA000AD231026A447F01127015227F09127007
:102FCA0015900536E0F532A3E0F533227D017F0145
:102FDA00124FE5227D017F07124FE5227D017F0214
:102FEA00124FE522127015900536E0F532A3E0F58E
:0A2FFA0033227D017F01124FE52212
:104DAE00C2957FFF127002124D1E7F0712642950AA
:104DBE000512003E80031261B0D28C7F0812642966
:104DCE0050051243BA80FEC22B12698A9000D1E0C0
:104DDE00FF7C117D00125CE4125E5790000FE0B470
:104DEE000105122831801090000FE0FF640260046C
:104DFE00EFB40303123265123E15301E11E54270F8
:104E0E000DE52754A060077FA0126FC1C21E7D075B
:104E1E007F05124FE54002C200E552C3940A50BB13
:104E2E003015B8E533453270B2C231126A4480ABE8
:104BF700EF253EFFEE353DCF2401FDE43FFC22AF1C
:104C07005A7E00EF2403FDEE33FC22E53E255AF5DC
:104C170082E4353DF58322E540255AF582E4353FA8
:104C2700F58322E56F256DF582E4356EF583E0FFA8
:104C3700E56F256DF582E4356EF58322E55A24028A
:104C4700FFE433FE22E56C2401FFE433FEC3E56D88
:104C57009FEE6480F874809822EF2540FFEE353F81
:104C670022E55C2EF582E4355BF583E0FD227FF4D7
:104C77007E01126D66E56C25E0F56C756D01227598
:064C87003D1E753E602297
:106D6600EF1FAA0670011ED39400EA9400400BE4BC
:0A6D7600FDEDC394C850E90D80F74D
:016D800022F0
:105379008F5BE55BB401197D017F06124FE5500C87
:105389009000B1E0FF7C0D7D00125CE47884062278
:10539900E55BB402131253EB50439000B2E0FF7C7B
:1053A9000D7D20125CE48035E55BB404161253EBE5
:1053B900500C9000B4E0FF7C0D7D60125CE47884B1
:1053C900760622E55BB403197D027F06124FE5508C
:1053D9000C9000B3E0FF7C0D7D40125CE47884768C
:0A53E90001227D027F06124FE5222B
:104FE500BF0107900020E0FE8048BF020790002126
:104FF500E0FE803EBF0307900022E0FE8034BF0440
:1050050007900023E0FE802ABF0507900024E0FEFC
:105015008020BF0607900025E0FE8016BF07079099
:105025000026E0FE800CBF0807900027E0FE800206
:10503500E4FEBD0103EE1322BD0204EEA2E122BD92
:105045000304EEA2E222BD0404EEA2E322BD0504A0
:10505500EEA2E422BD0604EEA2E522BD0704EEA2FF
:07506500E622BD0802EE3354
:01506C002221
:101D8700124C86900100E0F55A124C12E0123A5EAE
:101D97001DB6011DEB021E20031E55041E8A051EDB
:101DA700BF061EF4071F24081F500900001F7A12E0
:101DB7004C12A3E0B40A15E55A124C45E545B507A0
:101DC7000BE4B506077D017F01021F38124C06E5BB
:101DD700456D7001EC6003021F7A124BF7C2297F31
:101DE70001021F4D124C12A3E0B40A15E55A124C1A
:101DF70045E545B5070BE4B506077D017F02021FE0
:101E070038124C06E5456D7001EC6003021F7A122B
:101E17004BF7C2297F02021F4D124C12A3E0B40AEE
:101E270015E55A124C45E545B5070BE4B506077DA0
:101E3700017F03021F38124C06E5456D7001EC6007
:101E470003021F7A124BF7C2297F03021F4D124C60
:101E570012A3E0B40A15E55A124C45E545B5070B40
:101E6700E4B506077D017F04021F38124C06E545DD
:101E77006D7001EC6003021F7A124BF7C2297F04D1
:101E8700021F4D124C12A3E0B40A15E55A124C4535
:101E9700E545B5070BE4B506077D017F05021F3849
:101EA700124C06E5456D7001EC6003021F7A124B78
:101EB700F7C2297F05021F4D124C12A3E0B40A1581
:101EC700E55A124C45E545B5070BE4B506077D0114
:101ED7007F06021F38124C06E5456D7001EC600362
:101EE700021F7A124BF7C2297F06021F4D124C12AE
:101EF700A3E0B40A14E55A124C45E545B5070AE4D0
:101F0700B506067D017F078028124C06E5456D70F2
:101F170001EC705F124BF7C2297F078029124C1220
:101F2700A3E0B40A0F124C12A3A3E070077D017F50
:101F370008024F5A124C06E5456D7001EC703412D9
:101F47004BF7C2297F08020FFB124C12A3A3E070C4
:101F570022124C12A3E024F96008147016E4FF0261
:101F670060777FF47E01126D667D5E7F021267D017
:031F77001243BA58
:011F7A002244
:101B8600753F1E7540B0900108E0F55A124C1EE0F4
:101B9600123A5E1BB8011BF0021C28031C60041CD1
:101BA60098051CD0061D08071D3B081D700900007E
:101BB6001D86124C1EA3E0B40A13124C43E546B52B
:101BC600070BE4B506077D017F01021D53AF5A12CC
:101BD6004C08E5466D7001EC6003021D86124C60F0
:101BE600124BFED2297F01021D6D124C1EA3E0B4DA
:101BF6000A13124C43E546B5070BE4B506077D010B
:101C06007F02021D53AF5A124C08E5466D7001EC77
:101C16006003021D86124C60124BFED2297F02021F
:101C26001D6D124C1EA3E0B40A13124C43E546B5D3
:101C3600070BE4B506077D017F03021D53AF5A1259
:101C46004C08E5466D7001EC6003021D86124C607F
:101C5600124BFED2297F03021D6D124C1EA3E0B467
:101C66000A13124C43E546B5070BE4B506077D019A
:101C76007F04021D53AF5A124C08E5466D7001EC05
:101C86006003021D86124C60124BFED2297F0402AD
:101C96001D6D124C1EA3E0B40A13124C43E546B563
:101CA600070BE4B506077D017F05021D53AF5A12E7
:101CB6004C08E5466D7001EC6003021D86124C600F
:101CC600124BFED2297F05021D6D124C1EA3E0B4F5
:101CD6000A13124C43E546B5070BE4B506077D012A
:101CE6007F06021D53AF5A124C08E5466D7001EC93
:101CF6006003021D86124C60124BFED2297F06023B
:101D06001D6D124C1EA3E0B40A12124C43E546B5F3
:101D1600070AE4B506067D017F078031AF5A124CEB
:101D260008E5466D7001EC7057124C60124BFED2FE
:101D3600297F078032124C1EA3E0B40A13124C43CB
:101D4600E546B5070BE4B506077D017F08024F5A45
:101D5600AF5A124C08E5466D7001EC7023124C60C8
:101D6600124BFED2297F08020FFB124C1EA3A3E0E2
:101D7600700E124C1EA3E024F870057F01126077E6
:011D8600223A
:04496A008C5B8D5C79
:10496E00055CE55C7002055B14F5828C83E0F970E2
:10497E0003024A11EF7005124C868009BF010675BD
:10498E003F1E7540B0302946EF7007E9654560025D
:10499E00C322BF0107E965466002C322E4FEEEC3EF
:1049AE00995029EF700F124C68E53E2E124C16E00E
:1049BE006D6002C322EF6401700F124C68E5402E49
:1049CE00124C22E06D6002C3220E80D2D322202927
:1049DE0033E4FEEEC3995029EF700F124C68E53E9A
:1049EE002E124C16E06D6016C322EF6401700F128A
:1049FE004C68E5402E124C22E06D6002C3220E8000
:044A0E00D2D322C31A
:014A12002281
:060FFB008F5BAB05AA04A8
:101001007D027F07124FE55011E55BB4050C8B8221
:101011008A83E0640570030212687D017F07124F25
:10102100E55011E55BB4050C8B828A83E0640670A0
:1010310003021268C22AEB24FFF582EA34FFF5832A
:10104100E0F55D8B828A83E0FFF55EA3E0F9F55F51
:10105100EF123A5E107101107802107F03108604BE
:10106100108D05109406109B0710A208000010A710
:10107100755C01D22A802F755C02D22A8028755CAA
:1010810004D22A8021755C08D22A801A755C10D29C
:101091002A8013755C20D22A800C755C40D22A808C
:1010A10005755C80D22AE924FE700302116924F8D7
:1010B100605C2409600302117BE55BB401059000CB
:1010C100208045E55BB40205900021803BE55BB4DF
:1010D10003059000228031E55BB404059000238074
:1010E10027E55BB40505900024801DE55BB406058A
:1010F1009000258013E55BB407059000268009E583
:101101005B64087077900027E0455CF0806EE55BDA
:10111100B401059000208045E55BB40205900021F3
:10112100803BE55BB403059000228031E55BB404AC
:10113100059000238027E55BB40505900024801D00
:10114100E55BB406059000258013E55BB4070590C7
:1011510000268009E55B64087022900027E0FFE526
:101161005CF4FEEF5EF08014E55BB4050D8B828AC2
:1011710083E0FFD22F122992C22AC22A202A030217
:101181001268E55BB40109900020E0FD7F208060DA
:10119100E55BB40209900021E0FD7F218052E55B0F
:1011A100B40309900022E0FD7F228044E55BB40492
:1011B10009900023E0FD7F238036E55BB4050990AB
:1011C1000024E0FD7F248028E55BB406099000251A
:1011D100E0FD7F25801AE55BB40709900026E0FD5C
:1011E1007F26800CE55BB4080C900027E0FD7F278B
:1011F1007E00126495126E60D2AF2029047F0180B7
:10120100027F02127015A229922F126A8CAD5DE441
:10121100FF1267D0AD5EE4FF1267D0E55FB4010451
:101221007D388007E55FB40A077D367F061267D0F7
:10123100E55BB4050312662D7D077F05124FE5506E
:101241000A200007C2307F03122ECA7D017F0112DE
:101251004FE54005C230122ECA7D017F02124FE5D3
:071261004005C230122ECA45
:011268002263
:024F5A008F5B6B
:104F5C00ED24FF922F126A8CE55B123A5E4F8501AD
:104F6C004F8A024F8F034F94044F99054F9E064F63
:104F7C00A3074FA80800004FAE900020802190009E
:104F8C0021801C9000228017900023801290002416
:104F9C00800D90002580089000268003900027E06B
:104FAC00F55CE55C6024755E01E4F55DE55C30E084
:104FBC0007AD5EE4FF1267D0E55CC313F55C055EDC
:104FCC00055DE55DC3940840E3227D187F021267FE
:084FDC00D07D537F021267D063
:014FE40022AA
:10642900C2AFD284C285BF070BC28600E580A2E253
:10643900922A8019BF080BC28600E580A2E3922A3E
:10644900800BBF0508C28600E58013922AD286D246
:0564590085D2AFA22A6C
:01645E00221B
:10475500C229D22DE4FF125B117D2E7F031267D093
:104765007D607F021267D07F031270023024FD2026
:1047750024FDE5456407703B7E017F50124C868F12
:10478500828E837407F07D01E53E2D124C16E5827D
:1047950024FFF582E58334FFF583E0F9EF2DF582FB
:1047A500E43EF583E9F00DBD08DED2297F647E0085
:1047B500126D667F081264295043302995D22DE485
:1047C500FF125B117D607F021267D07D327F06127A
:1047D50067D07D1E7F051267D0C22DE4FF125B11E5
:1047E5007C017D507B087F507E0112570D7F08129A
:1047F500642950097F327E00126D6680F07F647EE9
:0448050000126D66CA
:01480900228C
:0255C6008F5AFA
:1055C800900138E0F55BE55A7020E55B124C45E543
:1055D800456F7001EE70547460255BF582E4341EEB
:1055E800AF82F55D8F5E7F408024E55A6401703B91
:1055F800E55B124C45E5466F7001EE702E74B025E0
:105608005BF582E4341EAF82F55D8F5E7F10120079
:1056180016855E82855D83E0FFA3E0FD126EAE8F86
:0B5628005CE4FD124A137F50126FC1BA
:015633002254
:024A13008D6BA9
:104A150075F020EF900280123A52AF8285836E8F37
:104A25006FE0F56CD394005003024AB2E56C941024
:104A3500507BE56B7014124C75124C4C506F124C38
:104A45002A124AB3056D056D80EFE56B6401702A86
:104A5500C201124C75124C4C5053124C2A124AB3D7
:104A6500302402800A30250C90000FE0B402057F47
:104A750050026FC1056D056D80DBE56B6402702D1D
:104A8500C201C202124C75124C4C5021124C2AA381
:104A9500E0FD12665D302402800A30250A90000F81
:0D4AA500E0B40203024173056D056D80DA77
:084AB20022A3E0FD12665D2263
:100D2E00855C82855B83A3A3E0FF855C82855B8304
:100D3E00A3222430F58274003EF583EDF0AF62EF0E
:100D4E003395E0FEE55F2FF582E55E3EF58322E505
:100D5E00822406F582E43583F583E0FF126E89ADB9
:100D6E0007AF63EF3395E0FEEF22A3A3E0FFE55C50
:100D7E002404F582E4355BF583E022E55F2405F576
:100D8E0082E4355EF583E022E55F2405F582E435E5
:100D9E005EF583E0FFE55F2406F582E4355EF583BC
:100DAE00E0228E69F56AAF68EF3395E0FEE5662FB7
:100DBE00F582E5653EF583222455F582E4340AF585
:100DCE0083EFF0E56275F007A422AF60EF3395E094
:100DDE00FEE56175F008900158123A52E5822FF542
:100DEE0082E5833EF58322E5662405F582E43565CA
:100DFE00F583E022E55E75F007A42454F582E43411
:100E0E000AF58322A3A3A3E0FF8D828C83E58224BF
:100E1E0004F582E43583F583E022E55E75F007A4E0
:100E2E002451F582E4340AF5832224E0F582740A13
:100E3E003EF583E5822DF582E5833CF58322E55E62
:100E4E0075F007A42453F582E4340AF58322E55F96
:100E5E002405F582E4355EF583E0FFE55F2406F5B3
:100E6E0082E4355EF583E022E55E75F007A4245238
:100E7E00F582E4340AF58322749F2562F582E43408
:100E8E0000F58322746F2562F582E43400F5832227
:100E9E002450F582E4340AF58322ECFF3395E0FE0C
:100EAE00EF25E0FFEE33FE75F02022E5602405F518
:100EBE0082E4355FF58322D3EF6480948022AB0702
:100ECE00AA068B828A83A3A3A3E0FFEB2404F582F8
:100EDE00E43AF583E0FD228F828E83A3A3A3E02262
:100EEE00855F82855E83A3A322AB5DAD5AAF5CAEF8
:100EFE005B22FFE562FD3395E0FCE55F2DF582E5B3
:100F0E005E3CF5832233CE33CE92E022A2E0CE13A6
:100F1E00CE132275F00AA42DFDE5F03CFCE5662209
:100F2E00E5602405F582E4355FF583E022E5627520
:100F3E00F008900158023A52E55E75F007A4245568
:100F4E00F582E4340AF583E022AB5AAD5DAF5CAEB8
:100F5E005B22EF7C002563FDEC35628D82F58322EA
:100F6E00A3A3E0FFAD5A22540FF5657808AF03AE88
:100F7E0002EF08220564E564AE632275F020123A92
:100F8E0052E0FEA3E0FF22E0FAA3E0FB780CFFAEF6
:100F9E00020822E0FCA3E0FD7804FFAE040822E57F
:100FAE00632561F582E43562F58322E5662DF582CF
:100FBE00E5653CF58322E5662FF582E5653EF58312
:100FCE00222431F5827400222480F58274023EAF11
:100FDE0082222560F560E4355FF55F2285608285AB
:0D0FEE005F83228F828E83A3A3E0640A221A
:02055B008F5AB5
:10055D00C22AE4F542D223D22D125B117D4B7F02CC
:10056D001267D07D02E4FF1267D07D32E4FF12677F
:10057D00D07D607F021267D07D027F07124FE5505C
:10058D00057F04127002900528E0F536A3E0F537DB
:10059D007F03127002E55A7006A22492298009E5A4
:1005AD005AB40104A2259229E53745367005D22AA1
:1005BD00020A223029DFE55A7006A2249229800909
:1005CD00E55AB40104A22592292029EAE55A700BB7
:1005DD00755B1E755C6085455D800EE55AB401093D
:1005ED00755B1E755CB085465DE55DD3940050036B
:1005FD00020A1C855C82855B83E0640B6003020A42
:10060D0017A3E0FFB40A0AE55DB40205D22A020A77
:10061D001CEF6401701E120D38A3E0640A7015E51D
:10062D005D6405700F120D38120D78120A4D1231DE
:10063D0038020A1C120D38E0B40111120D38A3E076
:10064D00B40109120EF7121725020A1C120D38E01B
:10065D006401701E120D38A3E064027015E55D642F
:10066D0005700F120D38120D78120A4D12629E028E
:10067D000A1C120D38E06401701D120D38A3E064E0
:10068D00037014E55DB4050F120D38120D78FDAB36
:10069D005A123A84020A1C120D38E0B4011D120DD3
:1006AD0038A3E0B40415E55DD39405400EAB5AAD07
:1006BD005CAC5BAF5D123004020A1C120D38E064B5
:1006CD0001701D120D38A3E064057014E55DB405CD
:1006DD000F120D38120D78FDAB5A125C03020A1C75
:1006ED00120D38E06401701D120D38A3E064067020
:1006FD0014E55DB4050F120D38120D78FDAB5A12CD
:10070D004ECD020A1C120D38E0B4011D120D38A396
:10071D00E0B40715E55DD39405400EAB5AAD5CAC66
:10072D005BAF5D12480A020A1C120D38E0640170BD
:10073D001D120D38A3E064087014E55DB4050F12A9
:10074D000D38120D78FDAB5A1262D8020A1C120D2B
:10075D0038E0B40215120D38A3E0B40A0DE55DB40E
:10076D000308AF5A12645F020A1C120D38E0B4027E
:10077D0016120D38A3E0B4010EE55DB40E09120E8C
:10078D00F9122D8E020A1C120D38E0B40216120D4C
:10079D0038A3E0B4020EE55DB40709120EF9125448
:1007AD006C020A1C120D38E0B40215120D38A3E0CC
:1007BD00B4090DE55DB40308AF5A1256A1020A1C27
:1007CD00120D38E064027019120D38A3E0B409114E
:1007DD00E55DB4040C120D38120F6E126876020A24
:1007ED001C120D38E064037021120D38A3E0640A69
:1007FD007018E55D64057012120D38120D78FD123A
:10080D006EAEAD5A1248BF020A1C120D38E06403D9
:10081D007029120D38A3E064017020E55DD39405B5
:10082D004019120D38120D78FD126EAE855A62AB5D
:10083D005DAD5CAC5B123EF6020A1C120D38E06435
:10084D00037021120D38A3E064027018E55D640594
:10085D007012120D38120D78FD126EAEAD5A126077
:10086D00F7020A1C120D38E0B40315120D38A3E07F
:10087D00B4030DE55DB40308AF5A126173020A1C8F
:10088D00120D38E0B40318120D38A3E0B40410E5CE
:10089D005DD394034009120F57124B5E020A1C12CE
:1008AD000D38E0B40315120D38A3E0B4050DE55D68
:1008BD00B40308AF5A126E9C020A1C120D38E0B434
:1008CD000316120D38A3E0B4060EE55DB40509124A
:1008DD000EF91269B0020A1C120D38E0640370198A
:1008ED00120D38A3E0B40711E55DB4040C120D38F8
:1008FD00120F6E126CBA020A1C120D38E0B40316F8
:10090D00120D38A3E0B4080EE55DB40409120EF91A
:10091D001269D5020A1C120D38E064057014E55DEC
:10092D00B4040F120D2EA3A3E0FDAB5A121F7B02D0
:10093D000A1C120D38E0B40516120D7CB40B10E52F
:10094D005DD394054009120F57123391020A1C1200
:10095D000D38E064067014E55DB4040F120D2EA37E
:10096D00A3E0FDAB5A12216D020A1C120D38E0B442
:10097D000616120D7CB40B10E55DD39405400912DB
:10098D000F571226A8020A1C120D38E06409701ABE
:10099D00120D38A3E0B40A12E55DB4040D120D3842
:1009AD00A3A3E0FF125EA0020A1C120D38E0640939
:1009BD007018120D38A3E0B40110E55DB4040B12EC
:1009CD000D38120F6E1263BB8045120D38E0B4095D
:1009DD0017120D38A3E0B4020FE55DD3940440085F
:1009ED00120EF71214D78027120D38E06409701A11
:1009FD00120D38A3E0B40310E55DB4040B120D38ED
:100A0D00120F6E125E0E80078000AF5A126CD72047
:100A1D002A030205A2C21ED22DAF5A125B117D60B0
:100A2D007F021267D07D327F031267D07F03127071
:0F0A3D0002125EE87FFF126FC1E47884F6C223D5
:080A4C0022FD126EAEAD5A222C
:081725008E5E8F5F8D608B6109
:10172D00120EE5FFE55F2404120D8DFD1265688F25
:10173D006274E22562F562C394005003021926E536
:10174D006294144003021926E5616406701D120DA2
:10175D0089B4010C120DD1120E9E7401F0021922E2
:10176D00120DD1120E9EE4F0021922E561640E6095
:10177D0003021844E55F240C120D8DFFB40A14E525
:10178D005F240D120D8DB40A0A120DD1120E2EE426
:10179D00F08013E55F240D120D8DFD126D2E120DCF
:1017AD00D1120E2EEFF0E55F240A120D8DFFB40A53
:1017BD0014E55F240B120D8DB40A0A120DD1120E11
:1017CD007CE4F08013E55F240B120D8DFD126D2E60
:1017DD00120DD1120E7CEFF0E55F2409120D8DFF75
:1017ED00640A6006EFD39409400A120DD1120E520D
:1017FD00E4F08010E55F2409120D8DFF120DD1125A
:10180D000E52EFF0120D89FFB40B15E55F24061291
:10181D000D8DB40B0B120DD1120E0874FFF0800854
:10182D00121952120E08EFF012192E120DC6120EC9
:10183D009E7401F0021922E561640A706E120DD1D9
:10184D00120E2EE4120DD0120E7CE4F0E55F240989
:10185D00120D8DFF640A6006EFD39409400A120D34
:10186D00D1120E52E4F08010E55F2409120D8DFFA8
:10187D00120DD1120E52EFF0120D89FFB40B15E5BA
:10188D005F2406120D8DB40B0B120DD1120E0874C0
:10189D00FFF08008121952120E08EFF012192E12D5
:1018AD000DC6120E9E7401F0021922E561640970D5
:1018BD0068120DD1120E2EE4120DD0120E7CE41210
:1018CD000DD0120E52E4F0120D89FFB40B15E55F29
:1018DD002406120D8DB40B0B120DD1120E0874FFD0
:1018ED00F08013E55F2406120D8DFD126D2E120D85
:1018FD00D1120E08EFF0E55F2407120D8DFFE55FA5
:10190D002408120D8DFD126D2E120DD1120DC61261
:10191D000E9E7401F0D22C8002C22CAF60126F9714
:10192D0022E55F2407F582E4355EF583E0FFE55F90
:10193D002408F582E4355EF583E0FD126D2EE56237
:10194D0075F007A422E55F2406F582E4355EF58384
:0C195D00E0FD126D2EE56275F007A4227B
:103138008F5E8D5FE55ED3941D5003023244E55ED9
:1031480094324003023244D22DAF5F125B117D46A8
:103158007F071267D0AF5E1235B874E2255EF55E60
:10316800120E2AE07021120E76E0701B120E4CE04F
:103178007015120E02E0700F120F46700A12325DBF
:103188007D537F0202323A12324CE55E75F007A495
:10319800120E9EE070047D3680027D387F0612672D
:1031A800D012324C120E28E0FFD394014034EF9431
:1031B80013502F7D097F061267D0120E2812325441
:1031C8007FF47E01126D667D0E7F031267D07D3518
:1031D8007F061267D07D097F061267D0120E76121D
:1031E80032547FF47E01126D66120E4CE0FF6005CA
:1031F800125BB4800A12325D7D0F7F031267D07DA7
:10320800277F021267D0120E02E0FFF46008126DE9
:10321800EB1235B880077D187F021267D07D377FA3
:10322800041267D0120F46FF126DEB1235B87D05F8
:103238007F061267D0C22DAF5F025B11C22CAF5F51
:10324800126F97227FF47E01126D6622E0FF126DE5
:0D325800EB1235B8227D187F021267D022DC
:02629E008D5E13
:1062A000EFD3941D402AEF9432502574E22FFFE47F
:1062B000FEEEFD3395E0FCEF75F007A42450F58267
:1062C000E4340A120E3FE4F00EBE07E5D22C800241
:0762D000C22CAF5E126F97B4
:0162D70022A4
:062D8E008E5E8F5F8D6078
:102D9400D22B120EE5FFE55F2404120DA7122EB507
:102DA400C39418501C855F82855E83A3A3A3E0FFB0
:102DB400E55F2404120DA7FD126E767882A60780C3
:102DC40006E47882F6C22B120D96122EB5C3943CFB
:102DD400500D120D96FD126E767883A6078006E4D8
:102DE4007883F6C22BE55F2407120DA7FF126F2923
:102DF4008F61E561D394004017E56194085011E5B3
:102E04005F2407120DA7FF126F29787FA60780069B
:102E1400787F7601C22BE55F2408120DA7FFE55FDA
:102E24002409120DA7122EBE401FE56194205019EB
:102E3400E55F2408120DA7FFE55F2409120DA7FD25
:102E4400126E767887A607800678877601C22BE50E
:102E54005F240A120DA7FFE55F240B120DA7122EA3
:102E6400BE401FE561940D5019E55F240A120DA7B9
:102E7400FFE55F240B120DA7FD126E767880A6077E
:102E8400800678807601C22BE55F240C120DA7FF23
:102E9400E55F240D120DA7FD126E767881A607302A
:102EA4002B07125A08D22C8002C22CAF60126F97E3
:102EB40022FD1265688F61E56122FD1265688F61EC
:062EC400E561D394002239
:06546C008E5E8F5F8D6073
:10547200D22B120EE5FFE55F2404120E6D1254D7F3
:105482009418501C855F82855E83A3A3A3E0FFE589
:105492005F2404120E6DFD126E767882A6078006D6
:1054A200E47882F6C22B120E5C1254D7943C500D53
:1054B200120E5CFD126E767883A6078006E478836E
:1054C200F6C22B302B07125A08D22C8002C22CAF04
:0454D20060126F975E
:0B54D60022FD1265688F61E561C322B2
:106F2900120EC54008EF6480948A5001227F002226
:106E7600AE05126F29EFC454F0FDAF06126F29EF6D
:036E86004DFF229B
:10645F008F5ED22D125B117D1E7F081267D07D26B5
:10646F007F081267D07D527F041267D0C22B12694A
:10647F008A125D7A787FE6FF125BB4125ABBC22D87
:06648F00AF5E125B11225A
:106876008D5EEFD3940A4006EFD3940F4003EF707A
:106886000E90002BEFF0D22CAF5E126F97D322C280
:086896002CAF5E126F97C322C4
:0256A1008F5E1A
:1056A300D22D125B117D207F051267D07D2E7F03E3
:1056B3001267D07D527F041267D090002BE0F55F14
:1056C300E55FB40B067D5F7F078034E55FB40C06AE
:1056D3007D5E7F068029E55FB40D067D0A7F02802B
:1056E3001EE55FB40E067D327F028013E55FB40FC3
:1056F300067D467F028008E55F70077D0A7F0312FF
:0957030067D0C22DAF5E125B11EC
:01570C00227A
:106CBA008D5E120EC5400EEF6480948650071265F1
:0D6CCA0000D22C8002C22CAF5E126F972208
:0269B0008D5EFA
:1069B200120ECC126568120EC54010EF648094A1CD
:1069C2005009900029EFF0D22C8002C22CAF5E1247
:0269D2006F97BD
:0169D40022A0
:0269D5008D5ED5
:1069D700120ECC126568120EC54010EF648094A1A8
:1069E7005009900028EFF0D22C8002C22CAF5E1223
:0269F7006F9798
:0169F900227B
:106E8900D3EF648094814008EF6480948A50012292
:036E99007F002255
:106F3900120EC54008EF648094A15001227F0022FF
:0814D7008E5E8F5F8D608B615A
:1014DF00120EE514F56374FC2561F5616403600F6A
:1014EF00E56164076009E561640B60030216C2C31E
:1014FF00E5636480948050030216C2E563648094B0
:10150F008840030216C2E4F562120D6F7803C333ED
:10151F00CE33CED8F92430F58274003EF583AF6216
:10152F00EF3395E0FE120DEAE4F00562E562B408D0
:10153F00D8756204E56164037029120D4B12170808
:10154F00120D6D7803C333CE33CED8F9120D40A3ED
:10155F00A3120D687803C333CE33CED8F9120FCF51
:10156F000216B9E56164077069120D4B1217081264
:10157F000D6D7803C333CE33CED8F9120D40A3A32C
:10158F00120D687803C333CE33CED8F9120FCF12B2
:10159F000D46A3A3A3120D687803C333CE33CED861
:1015AF00F92432F5827400120D461216CAC333CED7
:1015BF0033CED8F92433F5827400120D46120D5D27
:1015CF007803C333CE33CED8F92434F582740002B6
:1015DF0016B9E561640B60030216C2120D4BE012DF
:1015EF000F00A3E0FD126568126F39120D6D7803BD
:1015FF00C333CE33CED8F9120D40A3A3120D6878A2
:10160F0003C333CE33CED8F9120FCF120D46A3A397
:10161F00A3120D687803C333CE33CED8F92432F535
:10162F00827400120D461216CAC333CE33CED8F9C8
:10163F002433F5827400120D46120D5D7803C33307
:10164F00CE33CED8F92434F5827400120D46E582DC
:10165F002407120D617803C333CE33CED8F9243566
:10166F00F5827400120D46E5822408120E1F120F28
:10167F0000E5822409120E1FFD126568126F3912E0
:10168F000D6D7803C333CE33CED8F92436F582747B
:10169F0000120D46E582240A120D617803C333CE82
:1016AF0033CED8F92437F58274003EF583EDF0D2AE
:0A16BF002C8002C22CAF60126F975E
:1016C90022E5822404F582E43583F583E0FFE562AF
:1016D900FD3395E0FCE55F2DF582E55E3CF583E59C
:1016E900822405F582E43583F583E0FD12656812ED
:1016F9006F39AD07AF63EF3395E0FEEF780322E072
:10170900FFE562FD3395E0FCE55F2DF582E55E3C82
:0C171900F583A3E0FD126568126F392211
:045E0E008D5EAC07F2
:105E1200D3EC648094804035EC64809489502EE405
:105E2200FDECFF3395E0FEEF7803C333CE33CED8DB
:105E3200F92428F58274003EF583EDFF3395E0FEE8
:105E4200120DEAE4F00DBD08D8D22C8002C22CAFAC
:045E52005E126F97D6
:015E56002229
:1063BB008D5E120EC5402FEF648094895028EF1428
:1063CB00FFE55E24FF922B1250F4D22DAF5E125BD1
:1063DB00117542017F327E00126D66E54270FCC280
:0763EB002DAF5E125B1122D1
:08480A008F5E8C5F8D608B61F5
:10481200856082855F83120E12FD1265688F62E5E4
:1048220062D3940050030248B7E562943340030216
:1048320048B7E55E64067036D22DAF61125B117D1A
:10484200527F051267D0AF621235B8120F2EB40133
:104852000A120E867401F07D388007120E86E4F08B
:104862007D367F061267D0C22DAF61025B11E56013
:104872002406120F32640B703C120F2EB401081280
:104882000E867401F08005120E86E4F074F9255E3E
:10489200F55E75F004123998AFF0EF7014E56024FC
:1048A20006FBE4355FFAAD62E4FF1234B8D22C8025
:0C48B20006C22C8002C22CAF61126F976E
:0148BE0022D7
:083004008F5E8C5F8D608B6113
:10300C00856082855F83120E12FD1265688F62E502
:10301C0062D394005003023130E5629429400302DC
:10302C003130E55E64067037D22DAF61125B117DD5
:10303C00527F051267D0AF621235B8120EB9E0B4E8
:10304C00010A120E927401F07D388007120E92E480
:10305C00F07D367F061267D0C22DAF61025B11E5A1
:10306C00602406120EBDE0640B6003023130120EB8
:10307C00B9E0B40108120E927401F08005120E92A0
:10308C00E4F0E4FFFEE5602407120EBDE5822E128B
:10309C000E1FB40B04AF0680040EBE08E8EF7003DD
:1030AC00023130C39408507C120F3BEFF07E01EFDD
:1030BC002401FDE433FCEEC39DEC6480F87480982D
:1030CC005020E5602406120EBDE5822E120E1FFD67
:1030DC00120F3BE5822EF582E43583F583EDF00E7D
:1030EC0080CDE5602408120EBDE5822F120E1F6400
:1030FC000B602DEF2408FEC3E55E9EF55E75F004B3
:10310C00123998AEF0EE701CE5602407FDE4355FD3
:10311C00FC7E00ED2FFBEE3CFAAD627F011234B861
:0B312C00D22C8002C22CAF61126F9702
:013137002275
:0834B8008F638D648A658B6649
:1034C000756801E4F567120DB4E0FF6409703E12FF
:1034D00035A98003120F13D8FB120DB012359B785B
:1034E00008EF088003120F13D8FB120DB0A3A3E05E
:1034F000FFE568FD3395E0FCE5662DF582E5653C6A
:10350000F583A3A3A3E0FD126EAE023554120DB4F1
:10351000E0FF1235A98003120F13D8FB120DB01271
:10352000359B7804EF088003120F13D8FB120DB0FF
:10353000A3A3E0FF126FF8EF426AAE69AF6A7804A6
:10354000EF088003120F13D8FB120DB0A3A3A3E062
:10355000FF126FF8EF426AE563700FAF67120D71EB
:10356000120EAFE564900AC08012E563B40117AF94
:1035700067120D71120EAFE564900530120DE7E58C
:1035800069F0A3E56AF074042568F5680567C3E58A
:0A359000676480949050030234C673
:10359A0022A3E0FF126FF8EF426AAE69AF6A221205
:0E35AA006FF87569008F6AAE697804EF082229
:0A6FF800EFD3940940037F0022222A
:023A84008B5E57
:103A86001265688F61E561D394005003023B66E5D9
:103A96006194334003023B66D22DAF5E125B117D0B
:103AA600527F051267D0AF611235B8746F25611267
:103AB6000E96E060047D3880027D367F061267D060
:103AC6007F2C7E01126D66E561120F3DE0F55F7099
:103AD600077D1B7F061267D07D577F021267D0E5F0
:103AE6005F603B756001AF5F120D712401FFE43E1C
:103AF600FEAD60ED3395E0FCC3ED9FEE6480F8EC1F
:103B06006480985019120DD8E0B40A04E4FD8006CA
:103B1600120DD8E0FDE4FF1267D0056080C87F2C47
:103B26007E01126D66E561900530120F89900000E6
:103B3600EEF0A3EFF04E70077D1B7F061267D07D77
:103B46000C7F031267D0900000E07002A3E06009CA
:103B5600E56114FD7F01122AF0C22DAF5E025B11F2
:073B6600C22CAF5E126F9745
:013B6D002235
:024ECD008B5EFA
:104ECF001265688F5FE55FD394004077E55F943399
:104EDF005071D22DAF5E125B117D527F051267D0DC
:104EEF00AF5F1235B8749F255F120E8AE060047DA4
:104EFF003880027D367F061267D07F2C7E01126DBF
:104F0F00667F2C7E01126D66E55F900AC0120F89D5
:104F1F00900000EEF0A3EFF04E70077D1B7F06129E
:104F2F0067D07D0C7F031267D0900000E07002A362
:104F3F00E06009E55F14FDE4FF122AF0C22DAF5EB9
:0A4F4F00025B11C22CAF5E126F97D7
:014F59002235
:0262D8008B5EDB
:1062DA00126568AD07EDD394004025ED9433502044
:1062EA00E4FC120EA8ED900AC0120DE7E4F0A3F048
:1062FA000CBC10EE749F2D120E8AE4F0D22C800290
:07630A00C22CAF5E126F9779
:016311002269
:025C03008B5EB6
:105C0500126568AD07EDD394004036ED94335031FD
:105C1500E4FC120EA8ED900530120DE7E4F0A3F0B8
:105C25000CBC10EE746F2D120E96E4F0FCECFF33F5
:105C350095E0FEED120DE1E4F00CBC08F0D22C80ED
:085C450002C22CAF5E126F9742
:015C4D002234
:042AF0008F628D6301
:102AF400E4F564E5627052AF64120D7125E0FDEEF9
:102B040033FCAF63120D717805C333CE33CED8F9DD
:102B1400120E38120F958003120F1AD8FB120F757C
:102B24008003120F1AD8FB540FF566AF63120D71B0
:102B34007805C333CE33CED8F9120E38120FA180E4
:102B440003120F1AD8FB022BAEE56264017064AF66
:102B540064120D7125E0FDEE33FCAF63120D717844
:102B640005C333CE33CED8F92450F5827405120E42
:102B74003E120F958003120F1AD8FB120F758003B3
:102B8400120F1AD8FB540FF566AF63120D71780556
:102B9400C333CE33CED8F92450F5827405120E3ED9
:102BA400120FA18003120F1AD8FB540FF567ED54CE
:102BB4000FF568E565700CE5667008E5677004E577
:102BC40068607CAD65E4FF1267D0AD66E4FF126710
:102BD400D0E56564097045856769AF69FE7804EFDF
:102BE400088003120F13D8FBF569E5684269E569AB
:102BF400B4990B7D09E4FF1267D07D098027E5694C
:102C040075F00A84F56AFDE4FF1267D0E56A75F091
:102C14000AA4FFC3E5699FF56AFD8009AD67E4FF77
:102C24001267D0AD68E4FF1267D07FF47E01126DA5
:0F2C3400660564C3E564648094A05003022AF728
:012C4300226E
:10656800EFD394004015EF940B5010EFC3940A50EA
:1065780008EF75F00AA4FE8002E4FEEDD394004013
:106588000EED940B5009EDC3940A5003ED2EFEAFA7
:0165980006FC
:0165990022DF
:064B5E008E5E8F5F8B608C
:104B6400756105756240D3ED64809484407CED6486
:104B74008094A55075ED24FDF563D39404406BE552
:104B84006320E06613F5640562E562AE61700205B8
:104B94006114F5828E83E564F07403255FF55FE4A8
:104BA400355EF55EE4F563E563C395645033855F74
:104BB40082855E83E0FFA3E0FD126EAE0562E562CE
:104BC400AC617002056114F5828C83EFF0055FE53A
:104BD4005F7002055E055FE55F7002055E05638038
:104BE400C6D22CAF60126F97D322C22CAF60126F63
:024BF40097C365
:014BF600229C
:043EF6008C5F8D60F0
:103EFA00120EC55003023FCEEF6480949540030230
:103F0A003FCEEB648094875003023FCEEB648094EB
:103F1A00E44003023FCE120D717805C333CE33CE8F
:103F2A00D8F9120FD6F5638F64EB24FBF565D394A9
:103F3A00025003023FCEE56575F00384E5F06003A5
:103F4A00023FCEE56575F00384F567C3941050749B
:103F5A00120F827002056314F5828E83E567F0748E
:103F6A0005120FE0E4F565E565C395675052120F37
:103F7A00EAE0F566B40A10120F827002056314F5BE
:103F8A00828E83E4F0800F120F827002056314F5AB
:103F9A00828E83E566F0120FEAA3E0FF120FEAA30E
:103FAA00A3E0FD126EAE8F66120F827002056314D3
:103FBA00F5828E83E566F07403120FE0056580A72B
:0B3FCA00D22C8002C22CAF62126F9755
:013FD50022C9
:0826A8008E5E8F5F8D608B6177
:1026B000C22B120FF160030227451228205003029B
:1026C0002740E5649408E56394075074C3E56064AB
:1026D00080948A506B120EEEA3E0F562B40106906E
:1026E0000520022795E562B402069005220227958F
:1026F000E562B40306900524022795E562B404065A
:10270000900526022795E562B40506900528022764
:1027100095E562B4060690052A022795E562B4079E
:102720000690052C022795E562B4080590052E80D9
:1027300064E562B40905900530805AD22B02281155
:10274000D22B022811120EEEE064017052AD60AF80
:102750005FAE5E1228205003022811E5649408E55C
:102760006394074003022811C3E5606480948A40A3
:1027700003022811120EEEA3E0F562B40A059005DB
:10278000328012E562B401059005348008E562B438
:102790000209900536E563F0A3806FD22B80721298
:1027A0000EEEE06402706AAD60AF5FAE5E125C4E2A
:1027B0007563008F64C3E5649463E56394005051CE
:1027C000C3E560648094885048120EEEA3E0F56281
:1027D000B40107900538EFF08037E562B402059048
:1027E00005398026E562B4030590053A801CE56250
:1027F000B4040590053B8012E562B4050590053CE4
:102800008008E562B4060890053DE564F08002D2D8
:0F2810002B302B04C22C8002D22CAF61126F9799
:10281F0022124ABA8E638F64D3E564943BE56394C6
:02282F00002285
:064ABA008E658F66A90560
:104AC0007D057C00120FB9E0C3940A4005120FB9AE
:104AD000E4F00DBD00010CED640A4C70E7B9060767
:104AE000120DF5FF7E0022E964077010120DF575B6
:104AF000F00AA4ACF0FDE5662406801BE9640870AA
:104B000021120DF575F064A4ACF0FDE566240612E3
:104B10000DF9120F212407120DF92DFDE43CAF050C
:104B2000FE22E964097033120DF5FF7E007C037DDF
:104B3000E81239BAAC06AD07E5662406120DF97520
:104B4000F064120F242407120DF9120F2124081209
:0D4B50000DF92DFDE43CFEAF0522E4FEFF53
:014B5D002235
:065C4E008E658F66A905BA
:105C54007F057E00120FC4E0C3940A4005120FC4EE
:105C6400E4F00FBF00010EEF64084E70E7E964072B
:105C74007020E5662405F582E43565F583E075F06A
:105C84000AA4FFE5662406F582E43565F583E02F72
:045C9400FF227F006C
:015C980022E9
:083391008E5E8F5F8D608B6181
:10339900C22BD3E56064809484500302343FE56016
:1033A9006480948D400302343F120FF160030234AC
:1033B9003F120EE5123A5E33DF0133EA0233F503B9
:1033C90033FF04340905341306341D073427083440
:1033D90031090000343B756201756300D22B023458
:1033E90076756201756308D22B02347675620175B0
:1033F9006310D22B8077756201756318D22B806DAB
:10340900756201756320D22B80637562017563282B
:10341900D22B8059756201756330D22B804F75624A
:1034290001756338D22B8045756201756340D22BD3
:10343900803BC22B8037D3E56064809484402EE5BD
:10344900606480948D5026855F82855E83A3A3E0A6
:10345900B4011A855F82855E83A3A3A3E024F67075
:103469000A756201756358D22B8002C22B302B3743
:10347900E4FF120F60E4F00FBF08F7E56024FB8555
:103489006382856283F07F01E55F2404F582E43578
:103499005EF583E5822F120E1FFE120F60EEF00F0C
:0E34A900BF08E5D22C8002C22CAF61126F97D3
:0134B70022F2
:0448BF008F5E8D5F1C
:1048C300E55ED394005003024962E55E941540030C
:1048D300024962D22DAF5F125B117D5F7F051267C4
:1048E300D0AD5EE4FF1267D07D527F041267D07FA4
:1048F300F47E01126D6675F020E55E900280123A37
:1049030052AF828583628F63E0F560603DD394008C
:104913004046E56094105040E56025E0F560756120
:1049230001E5602401FFE433FEC3E5619FEE64808B
:10493300F87480985022120FADE0FF120FADA3E080
:10494300FD12665D0561056180D77D1B7F061267D9
:10495300D07D5F7F051267D0C22DAF5F025B11C2AE
:064963002CAF5F126F97FC
:01496900222B
:10216D008F5E8D5F8B60E55E640A7074E55FC3946E
:10217D000A40030222DA122310E4FDFF1267D0ADEC
:10218D005F1222E9E55F123A5E21B50121BB022102
:10219D00C10321C70421CD0521D30621D90721DF94
:1021AD000821E509000021EA90052002223490055E
:1021BD002202223490052402223490052602223474
:1021CD0090052802223490052A02223490052C0213
:1021DD00223490052E022234900530804A0222D3FB
:1021ED00E55E64017052E55FD394004006E55F94AF
:1021FD00034006E55F640A703C122310E55FB40AE4
:10220D000A7D0A1222E9900532801CE55FB4010AAD
:10221D007D0B1222F6900534800DE55FB402137D1F
:10222D000C1222F6900536E0FEA3E0FF1265CC02FB
:10223D0022E10222D30222DAE55E64026003022269
:10224D00E1E55FD3940050030222DAE55F94075075
:10225D007CD22DAF60125B117D277F081267D07D78
:10226D0006E4FF1267D07D14E4FF1267D0E55F240A
:10227D00FE601A14602114602814602F1460362437
:10228D000570437D0112230390053880307D0212C5
:10229D00230390053980267D0312232690053A806D
:1022AD001C7D0412232690053B80127D05122333DD
:1022BD0090053C80087D0612233390053DE0FF7E9E
:1022CD00001265FD800EAF60126CD78007C22CAF77
:1022DD0060126F97C22DAF60125B1122E4FF12677F
:1022ED00D07D527F041267D022E4FF1267D07D5259
:1022FD007F041267D022E4FF1267D07D527F041253
:10230D0067D022D22DAF60125B117D277F08126737
:10231D00D07D06E4FF1267D022E4FF1267D07D5214
:10232D007F041267D022E4FF1267D07D527F041222
:03233D0067D02244
:044C8D008E638F643F
:104C91000564E5647002056314F5828E83E0F566B0
:104CA100607AC3940850757F2C7E01126D66E4F51D
:104CB10065E565C395665064856482856383E0120A
:104CC1003A5E4CFE004CDC0A4CE00B4CE60C4CEC22
:104CD1000D4CF20E4CF80F00004D04E4FD802D7DCB
:104CE1005F7F0780287D5E7F0680227D0A7F0280AC
:104CF1001C7D327F0280167D467F0280107D0A7FF7
:104D010003800A856482856383E0FDE4FF1267D036
:0C4D11000564E56470020563056580958B
:014D1D002273
:061F7B008F5E8D5F8B609C
:101F8100C22BE55E640A600302206FE55F123A5ED0
:101F91001FB0011FC3021FD6031FE9041FFC052048
:101FA1001206202807203E082053090000206B124A
:101FB10020A47D011220F2756101756200D22B020D
:101FC100208B1220A47D021220F275610175620836
:101FD100D22B02208B1220C07D031220FF756101DC
:101FE100756210D22B02208B1220C07D041220FFBB
:101FF100756101756218D22B02208B1220DC12212F
:10200100527D05122122756101756220D22B0220B9
:102011008B1220DC1221527D06122122756101757D
:102021006228D22B02208B12210C1221667D07120D
:10203100212F756101756230D22B02208B12210C88
:102041001221667D0812212F756101756238D22B2C
:10205100803812213CE4FDFF1267D07D091221591D
:10206100756101756240D22B8020C22B801CE55E18
:1020710064017016E55F24F6701012213C7D0A128E
:102081002159756101756258D22B302B09AF62AEAF
:1020910061124C8D8005AF60126CD7C22DAF6012FA
:0220A1005B11D1
:1020A30022D22DAF60125B117D577F021267D07D64
:1020B30005E4FF1267D0E4FDFF1267D022D22DAFF3
:1020C30060125B117D577F021267D07D05E4FF121A
:1020D30067D0E4FDFF1267D022D22DAF60125B11EF
:1020E3007D577F021267D07D05E4FF1267D022E49B
:1020F300FF1267D07D527F041267D022E4FF12677C
:10210300D07D527F041267D022D22DAF60125B11B3
:102113007D577F021267D07D05E4FF1267D022E46A
:10212300FF1267D07D527F041267D022E4FF12674B
:10213300D07D527F041267D022D22DAF60125B1183
:102143007D577F021267D07D05E4FF1267D022E43A
:10215300FDFF1267D022E4FF1267D07D527F041285
:0A21630067D022E4FDFF1267D022CE
:1035B8008F72E572D3945940107D5A12369F24A613
:1035C800FD700302369E023699E572D3944F401679
:1035D800E572945A50107D5012369F24B0FD700346
:1035E80002369E023699E572D394454016E57294E8
:1035F8005050107D461236A724BAFD700302369E3D
:10360800023699E572D3943B4012E5729446500C09
:103618007D3C1236A724C4FD607C8075E572D39486
:10362800314012E572943C500C7D321236AF24CEF4
:10363800FD6063805CE572D394274012E572943292
:10364800500C7D281236AF24D8FD604A8043E572BD
:10365800D3941D4016E572942850107D1EE4FF1285
:1036680067D0E57224E2FD602D8026E572D39413BD
:103678004016E572941E50107D14E4FF1267D0E5E1
:103688007224ECFD60108009E572C394145007ADF4
:1036980072E4FF1267D022E4FF1267D0E57222E4D9
:0F36A800FF1267D0E57222E4FF1267D0E57222AD
:105B11008F6AE56A700C302D097F011270157FC004
:105B2100801FE56A700C202D097F011270027FC071
:105B31008026E56AB40112302D0F7F021270157FA5
:105B410030120016C22F026A8CE56AB40114202DAE
:105B5100117F021270027F30126FC17FC87E001266
:035B61006D66224C
:106A68008F69D22D125B117D607F021267D07D3253
:106A78007F061267D07D1E7F051267D0C22DAF69D1
:046A8800125B11226A
:106CD7008F69D22D125B117D607F021267D07D30E4
:0D6CE7007F031267D0C22DAF69125B11222E
:0E6F97008F68302C03026A68AF68126CD72234
:105EA000EF24FE60101460162402701C7F01127033
:105EB000157F8080107F021270157F2080077F037E
:105EC0001270157FA01200167FF47E01126D6675A8
:105ED0004204E54270FC7F647E00126D667F03120F
:085EE00070027FA0126FC122C5
:1065FD008E618F627C007D0A1239CCAD07E4FF12EB
:10660D0067D07D5B7F061267D0AE61AF627C007D87
:10661D000A1239CCE4FF1267D07D4A7F070267D09A
:0465CC008E618F62EB
:1065D0007C007D3C1239CC1235B87D057F061267F0
:1065E000D0AE61AF627C007D3C1239CCED4C600CCA
:0C65F000AF051235B87D4A7F071267D056
:0165FC00227C
:0260F7008D5EBC
:1060F900120EC5402FEF648094955028120D7178C7
:1061090005C333CE33CED8F9120FD6FEE4FD0FEF17
:10611900AA0670010E14F5828A83E4F00DBD20EE03
:0B612900D22C8002C22CAF5E126F97D8
:016134002248
:106173008F5E900540E0D394024015D22D125B113F
:106183007542037F327E00126D66E54270FC801516
:10619300D22DAF5E125B117D1B7F061267D07D0C83
:0D61A3007F031267D0C22DAF5E125B112288
:106E9C007E10900540E4F0A3DEFC7E10D22C126F25
:016EAC00974E
:016EAD0022C2
:106EAE00BF0A02E4FFBD0A02E4FDEF75F00AA42D4D
:026EBE00FF22B1
:106D2E00EFD394094002E4FFEDD394094002E4FD51
:0C6D3E007804EF08800123D8FD4DFF22EF
:1040A90007010203040506070707060504030201C1
:1040B90003010A0A030307050303020503020A0AA7
:1040C90004050A0A0104050A0A0A04050A0A020380
:1040D900070A0A03040A0A04024B00020032072EE7
:1040E90003024B0002003202055F000302055F0074
:1040F9000402055F000502055F000604072E082675
:104109000640033204072E08260640025304081EFF
:1041190008260452010008024B00020032072E084B
:104129001E08260452010003072B02350636030731
:104139002B0235063803072B0235072603072B0206
:1041490035025302055F000F02055F001002055F8B
:10415900001102055F001202055F001302055F00EE
:0A41690014080C0A1D020500241BB7
:1053F3007461F0A37420F0A37452F0A37401F0A3BA
:1054030022A3F0A37461F0A37440F022F0A3740309
:10541300F0E4A3F0A37410F0A37403F0E4A3F0A3E7
:10542300227461F0A37441F0A3227461F0A3F0A38A
:105433007430F0A3227496F0A37432F0A37495F041
:10544300A3741EF0A322F0A37461F0A314F0A37459
:1054530070F0A3E4F022A3F0A37452F0A3223CF56E
:0954630083E0FEEF3395E0FC222A
:10003E007E407FA97C017D507B08125FF57E407F5C
:10004E00B17C017D587B08125FF57E407FB97C0143
:10005E007D007B04125FF57E407FC57C017D087BB1
:10006E0004125FF57E407FC17C017D107B04125F20
:10007E00F57E407FBD7C017D187B04125FF57E40CE
:10008E007FCE7C017D207B05125FF57E407FC97C93
:10009E00017D287B05125FF57E407FD37C017D308C
:1000AE007B05125FF57E407FD87C017D387B041284
:1000BE005FF57E407FDC7C017D407B04125FF57E28
:1000CE00407FE07C027DA07B09125FF57E407FE9D8
:1000DE007C027DC07B07125FF57E407FF07C027D47
:1000EE00E07B05125FF57E407FF57C037D007B058E
:1000FE00125FF57E407FFA7C037D207B05125FF553
:10010E007E407FFF7C037D407B05125FF57E417F45
:10011E00047C037D607B09125FF57E417F0D7C03BD
:10012E007D807B09125FF57E417F167C037DA07B6F
:10013E0009125FF57E417F1F7C037DC07B11125F2C
:10014E00F57E417F307C037DE07B07125FF57E41BB
:10015E007F377C047D007B07125FF57E417F3E7CFE
:10016E00047D207B07125FF57E417F457C047D4038
:10017E007B07125FF57E417F4C7C047D607B051210
:10018E005FF57E417F517C047D807B05125FF57E9D
:10019E00417F567C047DA07B05125FF57E417F5B1F
:1001AE007C047DC07B05125FF57E417F607C047D03
:1001BE00E07B05125FF57E417F657C057D007B054A
:1001CE00125FF57E417F6A7C057D407B09125FF5EB
:1001DE009000297417F07F0312650090002874199F
:1001EE00F090002074B1F09000217491F0900022F4
:1001FE007403F0900023747FF090002404F09000BC
:10020E00257403F0E4900026F0900027F090003063
:10021E00740912540F7415F0A37403F0A37415121D
:10022E00540F7409F0A37403F0E4FFEFFD3395E06F
:10023E00FC74302DF582740012546174102DF58209
:10024E0074003CF583EEF00FBF08E0E4FFEFFD33E2
:10025E0095E0FC74382DF582740012546174182DDB
:10026E00F58274003CF583EEF00FBF08E090052098
:10027E00E4F0A374B4F0900522E4F0A374B4F0900B
:10028E0005247401F0A374E0F0900526E4F0A37445
:10029E0078F09005287402F0A37458F090052AE4C3
:1002AE00F0A3743CF090052C7402F0A37458F07413
:1002BE000790052EF0A3F0900530F0A3F0900532D4
:1002CE00F0A3F0900534F0A3F0900536E4F0A3749B
:1002DE003CF0900538740AF09005397428F09005BA
:1002EE003A7405F090053B740AF090053CF09005C9
:1002FE003D7428F09000A47401F0900B607415F01A
:10030E00A37411F09000A57401F0900B807415F099
:10031E00A37410F09000A67401F0900BA07415F069
:10032E00A37421F09000A77401F0900BC07415F027
:10033E00A37420F09000A87401F0900BE07415F0F7
:10034E00A37431F09000A97401F0900C007415F0B4
:10035E00A37430F09000AA7401F0900C207415F084
:10036E00A37441F09000AB7401F0900C407415F042
:10037E00A37440F09000AC7401F0900C60745312B2
:10038E0053FD74361253FD7438F0A3E4F0A3745386
:10039E00F0A3E4F09000AD04F0900C80745312536F
:1003AE00FD7434F0A37421F0A37453F0A3E4F09021
:1003BE0000AF04F0900CC01253FB7430F0740312B3
:1003CE005459E4F09000B004F0900CE01253FB741A
:1003DE0030F07404125459E4F09000B104F0900D12
:1003EE00001253F374321253FD7452F0A37420F0C2
:1003FE009000B27401F0900D201253F37432F0A3FA
:10040E00740212545A7420F09000B37401F0900DDF
:10041E004074531253FD7433F0A3E4F09000B4040F
:10042E00F0900D601254247430F074021254049043
:10043E0000B57401F0900D801254247430F07405E0
:10044E001254049000B67401F0900DA0125424744E
:10045E0030F0A374061254059000B77401F0900D9D
:10046E00C01254241254387498F0A3744B125405CD
:10047E009000B87401F0900DE012542412543874A8
:10048E0093F0A374181254059000B97401F0900EF5
:10049E00001254247430F0A37413125405A3747014
:1004AE00F0A37402F09000BA14F0900E2012542DA6
:1004BE007412F0A374701253FD7461F0A314F090D3
:1004CE0000BB7401F0900E4012542D741112544959
:1004DE009000BC04F07461900E6012542F741412CC
:1004EE0054499000D104F09011001254247492F0EB
:1004FE00A3744BF0A37490F0A37402F0A37490F065
:10050E00A37432F07499A3F0A3F0A374601253FD98
:10051E0074911253FD7491F0A3E412540590000FE0
:10052E007401F0125EE87F011270157F4012001602
:10053E007D2F7F071267D07D0C7F031267D07D322F
:0C054E007F061267D07D1E7F051267D06B
:01055A00227E
:0A5FF5008E5A8F5B8C5C8D5D8B5E15
:105FFF00E4F9C3E55E6480F8E96480985028E9FF0E
:10600F003395E0FEE55B2FF582E55A3EF583E49389
:10601F00FFE9FD3395E0FCE55D2DF582E55C3CF590
:06602F0083EFF00980CCB4
:016035002248
:10577300AF6AEF3395E0FEE56975F008A42428F5D8
:1057830082E43400F583E5822FF582E5833EF583D9
:10579300E0FFE56AFD3395E0FC22AB66AD65AF64DF
:1057A300223EF583E0FD74B82FF582741D3EF58328
:1057B300EDF0056AE56A22EF3395E0FEEF25E0FFA1
:1057C300EE33FE22A2E0CE13CE13223CF583EFF09C
:0557D300056AE56A22F1
:045C99008C5B8D5C37
:105C9D00EF6043D201D202D20CE4F55D855C8285C2
:105CAD005B83E0FEA3E04E6027AF5D1257BAE55C63
:105CBD002FF582E55B3EF583E0FEA3E0FF12453252
:105CCD00922920290B055DC3E55D6480949040CC3D
:065CDD00C201C202C20C6C
:015CE300229E
:045CE4008C608D61E2
:105CE800EF6043D201D202D20CE4F562856182856D
:105CF8006083E0FEA3E04E6027AF621257BAE56109
:105D08002FF582E5603EF583E0FEA3E0FF12453201
:105D1800922D202D0B0562C3E5626480949040CCDF
:065D2800C201C202C20C20
:015D2E002252
:04453200AD07AC061F
:10453600C22E780CEF0880031257C7D8FB540FF52C
:10454600637808AF05AE04EF0880031257C7D8FB9F
:10455600540FF5647804AF05AE04EF0880031257D4
:10456600C7D8FB540FF565ED540FF566E56360712A
:10457600B4010812579D123D348066E563B4020803
:1045860012579D126C428059E563B4030812579D79
:104596001238AA804CE563B4040812579D126BE3E7
:1045A600803FE563B4050812579D1224FA8032E570
:1045B60063B4060812579D1212698025E563B40795
:1045C6000812579D12527D8018E563B408081257E9
:1045D6009D1259AD800BE563B4090612579D126909
:0345E600FAA22E08
:0145E90022AF
:103D34008F678D688B69E567B40113900020E0FFFD
:103D4400125A63900020EFF0FD7F20023DF1E567F9
:103D5400B40211900021123DF7900021EFF0FD7F95
:103D640021023DF1E567B40311900022123DF79062
:103D74000022EFF0FD7F22023DF1E567B4041090CC
:103D84000023123E01900023EFF0FD7F23805EE5C7
:103D940067B40516900024123E01900024EFF0FD54
:103DA4007F247E0012649502662DE567B4061090A8
:103DB4000025123E0B900025EFF0FD7F25802EE5B7
:103DC40067B40710900026123E0B900026EFF0FD1A
:103DD4007F268019E567B40819900027E0FFAB69D6
:103DE400AD68125A63900027EFF0FD7F277E001222
:103DF400649522E0FFAB69AD68125A6322E0FFAB21
:103E040069AD68125A6322E0FFAB69AD68125A6368
:013E1400228B
:105A6300D22FAC07BD01047E018033BD02047E0248
:105A7300802CBD03047E048025BD04047E08801EA3
:105A8300BD05047E108017BD06047E208010BD076F
:105A9300047E408009BD08047E808002C22FBB01C2
:105AA30005EE4204800BEB7006EEF452048002C252
:075AB3002F302F03AF042286
:015ABA0022C9
:026C42008B675E
:106C4400C22FEF7016ED7013E5677003025D7AE5ED
:0B6C540067B40107787FE6FF125BB415
:016C5F002212
:0638AA008F678D688B6939
:1038B000E5677007123990E4FD801AE567B40107E7
:1038C0001239907D01800EE567B4020CAD69AF68D6
:1038D000126FA57D02024A13E567B4030612417315
:1038E000C21E22E567B40415AD69AF681265688F22
:1038F00043754205E542700302398F80F7E567643E
:10390000067017E5687013F56A12577374102DF579
:103910008274001257CEB408F022E567640770176E
:10392000E5687013F56A12577374182DF5827400E8
:103930001257CEB408F022E56764087027E5687076
:1039400023E569701FF56AAF6AEF3395E0FE7410E6
:103950002FF58274001257A4B408EC754201E542B9
:10396000602D80FAE56764097025E5687021E569D6
:10397000701DF56AAF6AEF3395E0FE74182FF5827B
:0F39800074001257A4B408EC754201E54270FCC4
:09398F0022AD69AF68126FA52298
:106BE3008F67AE03AF05E567D394004012E5679462
:106BF30007500CAD06126FA5AD07AF6712682422CC
:1024FA008F678D688B69E5677018E5687014E56900
:10250A0070057F01126FC1E569640160030226A7A5
:10251A008043E567701CE568B40117E56970057FBB
:10252A0004126FC1E569640160030226A77F0402F1
:10253A0026A4E5677029E56864027023E5697005D9
:10254A007F05126FC1E569640160030226A7900046
:10255A000FE0B403057F010226A47F050226A4E545
:10256A0067B4011BE5687017E56970057F02126F91
:10257A00C1E569640160030226A77F020226A4E579
:10258A0067B4011CE568B40117E56970057F081294
:10259A006FC1E569640160030226A77F080226A4C9
:1025AA00E56764017029E56864027023E5697005CE
:1025BA007F0A126FC1E569640160030226A79000D1
:1025CA000FE0B403057F020226A47F0A0226A4E5CF
:1025DA0067B4021BE5687017E56970057F40126FE2
:1025EA00C1E569640160030226A77F400226A4E5CB
:1025FA0067B4021CE568B40117E56970057F10121B
:10260A006FC1E569640160030226A77F100226A450
:10261A00E56764027024E5686402701EE569700566
:10262A007F50126FC1E5696401707290000FE0B4C7
:10263A0003047F4080647F508060E567B40317E538
:10264A00687013E56970057F80126FC1E5696401DE
:10265A00704B7F808044E567B40318E568B40113C2
:10266A00E56970057F20126FC1E5696401702E7FEC
:10267A00208027E56764037024E5686402701EE51C
:10268A006970057FA0126FC1E569B4011090000F4F
:0E269A00E0B403047F8080027FA012001622AD
:101269008F678D688B69E5677017AD69AF68126F15
:10127900A58E348F35D3E5359400E534940050F5C7
:1012890022E567B4011BE568B40116E5697007C278
:10129900307F01122ECAE569640160030214D68009
:1012A90058E5676401702BE56864027025E569708B
:1012B90007C2307F02122ECAE56964016003021475
:1012C900D690000FE0640370030214D6D2307F0277
:1012D9008031E5676401702EE56864037028E5696B
:1012E9007007C2307F03122ECAE5696401600302E8
:1012F90014D690000FE0B40306D2307F018004D2E7
:10130900307F03022ECAE5676401702DE568640425
:101319007027E569700CC2307F01122ECA7F401216
:101329006FC1E569640160030214D6D2307F0112EE
:101339002ECA7F40120016807CE5676401703AE589
:101349006864057034E569700CC2307F02122ECAD8
:101359007F10126FC1E569640160030214D6900021
:101369000FE0640370030214D6D2307F02122ECA32
:101379007F10120016D22F803EE5676401703BE5AD
:101389006864067035E569700CC2307F03122ECA95
:101399007F50126FC1E569640160030214D6D2302F
:1013A9007F03122ECA90000FE0B403047F4080022D
:1013B9007F50120016C22F026A8CE56764027029F9
:1013C900E56864017023E56970057F100214BDE5C5
:1013D90069B401057F100214C7E56964026003025C
:1013E90014D6D22F7F010214D3E56764027029E570
:1013F9006864027023E56970057F200214BDE56900
:10140900B401057F200214C7E56964026003021470
:10141900D6D22F7F020214D3E56764027029E568EA
:1014290064037023E56970057F400214BDE569B462
:1014390001057F400214C7E569640260030214D6FE
:10144900D22F7F030214D3E56764027023E5686431
:1014590004701DE56970047F808059E569B4010451
:101469007F80805AE56964027063D22F7F04805AB5
:10147900E56764027023E5686405701DE569700419
:101489007F048030E569B401047F048031E5696433
:1014990002703AD22F7F058031E5676402702EE52C
:1014A90068640670287D017F07124FE5401FE569D2
:1014B90070057F08027002E569B401057F080270B2
:0E14C90015E569B40207D22F7F061229922280
:06527D008F678D688B694C
:10528300E567703BE5687037E569700690000F04C9
:105293008021E569B4010A90000F7402F0D22F80D7
:1052A30047E56964027041C21E7FFF126FC190001F
:1052B3000F7403F0C2307F02122ECAD22F8029E569
:1052C3006764017023E568701F7D077F05124FE552
:1052D3005016E569700BC200C2307F03122ECA80DC
:1052E30007E569B40102D200302F0C90000FE0FDF6
:0752F3007F0F7E001264959D
:0152FA002291
:1059AD008F678D688B69E567700C1259F1749F2FA5
:1059BD00F58274008019E567B4010C1259F1749FDA
:1059CD002FF58274008016E567B402091259F93E6D
:1059DD00F583E4F022E567B403091259F93EF58326
:1059ED007401F022AD69AF68126FA522AD69AF6881
:0B59FD00126FA5746F2FF5827400225A
:0269FA008F67A5
:1069FC00AF057804EF08800123D8FD4BF568E567F7
:106A0C00B40908E568B4990302506DAD68AF67121C
:026A1C00665DB5
:016A1E002255
:0D6FA500EF75F00AA47C002DFFEC35F0FE26
:016FB20022BC
:046824008F688D6983
:10682800C3E569648094E4501BE4F56AC3E56964D0
:1068380080F8E56A648098500BC22FAF68122992DD
:04684800056A80E875
:01684C002229
:0D6FB300C296007F0512696412659AD2969D
:016FC00022AE
:106E4A00126FB3EF20E0F9C296007F06126964C29E
:066E5A00B60000D29622F2
:106E6000126FB3EF20E0F9C296007F04126964C28A
:066E7000B60000D29622DC
:046135008E608F6188
:10613900AE04AF058E638F64C296007F0312696453
:10614900E560FF126964AF61126964E4F562126582
:106159009AE5642562F582E43563F583EFF005621B
:09616900E562C3942040E7D296E0
:01617200220A
:085D2F008E658F668C678D689C
:105D3700126FB3EF20E0F985656A85666BC296003E
:105D47007F02126964E567FF126964AF68126964CC
:105D5700E4F569E56B2569F582E4356AF583E0FFCB
:105D67001269640569E569C3942040E7C2B600007B
:025D7700D296C2
:015D79002207
:0A570D008E5A8F5B8C5C8D5D8B5E05
:10571700C2AF126E4A126FB3EF20E0F9855C608565
:105727005D61C296007F02126964E55AFF126964DF
:10573700AF5B126964E4F55FAF5EEF3395E0FEC3DC
:10574700E55F9FEE6480F87480985014E561255FEB
:10575700F582E43560F583E0FF126964055F80D860
:0B576700C2B60000D296126E60D2AFF6
:015772002214
:106495008E6B8F6C8D6DC2AF126E4A126FB3EF208B
:1064A500E0F9C296007F02126964E56BFF12696428
:1064B500AF6C126964AF6D126964C2B60000D29602
:0664C500126E60D2AF224E
:1061B000C2AFE4F55BF55CF55DF55EF55FF55AAEF3
:1061C0005EAF5FAC5BAD5C1261357420255CF55C45
:1061D000E4355BF55B7420255FF55FE4355EF55EC5
:0B61E000055AE55AC3948940D6D2AF9F
:0161EB002291
:105EE800C2AF756200756300756400E4F560F56122
:105EF800F55F126E4AAE63AF64AC60AD61125D2FA0
:105F080074202561F561E43560F56074202564F539
:105F180064E43563F563055FE55FC3948940D31294
:045F28006E60D2AF26
:015F2C002252
:105837000500050105030507050F051F051E051CC6
:10584700051805100201040E040A03060101040BE2
:105857000304040F020304010302040D0200020201
:1058670003000409040403050307010003030407F5
:10587700030104060402040C0516051500000615AD
:0E588700062A060C06380633061E0612061701
:104E3E002430F58274003EF583EDFF3395E0FEE5F8
:104E4E00822FF582E5833EF583E0FFEDFB3395E09F
:104E5E00FA22AF41126964C29312700CD293D2AF90
:104E6E00223EF583E0FC74B82FF582741D3EF58367
:104E7E00ECF00D221528E528D394002225E02437E6
:104E8E00F582E43458F583E49322E4F57BD20EC226
:104E9E0027C21DC21A227FA0126FC1E4F542C21EA4
:104EAE002212700CD2B67801EF0822122C44D2CA0C
:0F4EBE00D20ED22722ECFF3395E0FEEF780322CD
:10423900200E2F900540E004F576D36480948150D8
:10424900030242F9D3E5766480948F400375760FB3
:10425900900029E0FF122C4490002AE0F575124ED7
:104269009822301A58302712124E8240030242F91E
:10427900C2CAC227D21D85752822301D0A124E8254
:10428900506EC227C21D22AF791579EF700BC21A81
:10429900E57525E0F528D21D22E57A30E00585751A
:1042A900288008E57575F003A4F528AF7A7801EF41
:1042B90008800103D8FDF57AD227D2CA22D576081B
:1042C900C20EE4F542C21E22057B7440257BF582AD
:1042D900E43405F583E0124E8A540FF5797401939D
:1042E900F57A700AD21DE57525E025E0F528D21A80
:0142F90022A2
:1052FB00200E12900029E0FF122C4490002AE0F5BA
:10530B0077124E9822301A5130270F124E82505D71
:10531B00C2CAC227D21D85772822301D0A124E829F
:10532B00504BC227C21D22AF791579EF7007C21AF5
:10533B00C20EF54222E57A30E0058577288008E534
:10534B007775F003A4F528AF7A7801EF0880010395
:10535B00D8FDF57AD227D2CA22E543124E8AFA74C7
:0D536B000193FBEA540FF579EBF57AD21AA5
:015378002212
:10659A00E4F56FD297F56EC2B612700CAF6F780140
:1065AA00EF08800123D8FDF56F309703436F01127E
:1065BA00700CD2B6056EC3E56E6480948840D8AF7D
:0165CA006F61
:0165CB0022AD
:09700C0000000000000000002259
:10677900C2B7E4FEC2B612700CEF30E704D2B5809E
:1067890002C2B5124EAF800123D8FDFF12700C0E64
:0B679900BE08E1C2B6D2B7D2B6D2B53E
:0167A40022D2
:0D001600C2AFEF4227AF27126779D2AF22A9
:0E6FC100C2AFEFF45227AF27126779D2AF228A
:10696400E4FEC2B612700CEF30E704D2B58002C266
:10697400B5124EAF800123D8FDFF12700C0EBE0875
:05698400E1D2B6D2B51E
:0169890022EB
:09701500C2AFEF4241124E6022AD
:0A700200C2AFEFF45241124E6022BB
:102C4400EF123A5E2CAC012CB3022CBA032CC10453
:102C54002CC8052CCF062CD6072CDD082CE4092C17
:102C6400EB0A2CF20B2CF90C2D000D2D070E2D0E5A
:102C74000F2D15102D1C112D23122D2A132D311457
:102C84002D38152D3F162D46172D4D182D54192D61
:102C94005B1A2D621B2D691C2D6B1D2D721E2D7947
:102CA4001F2D802000002D6975CB8E75CAC6227534
:102CB400CB9575CA772275CB9B75CA692275CBA053
:102CC40075CABA2275CBA675CA332275CBAB75CA41
:102CD400632275CBB075CA022275CBB475CAA32220
:102CE40075CBB875CAFA2275CBBC75CAD82275CB18
:102CF400C075CAA82275CBC475CA362275CBC775F0
:102D0400CA862275CBCA75CABC2275CBCD75CAB426
:102D14002275CBD075CA762275CBD375CA3022758D
:102D2400CBD575CAB22275CBD875CA132275CBDA46
:102D340075CA522275CBDC75CA7D2275CBDD75CA86
:102D44006E2275CBE075CA542275CBE275CA1B227C
:102D540075CBE375CAC32275CBE575CA5E2275CB04
:102D6400E675CADA22801C75CBE875CA902275CB49
:102D7400EA75CAD92275CBEC75CA092275CBED75F3
:0A2D8400CA292275CBE875CA412266
:10002600C3EF648094A15008EF25E025E0F528226F
:04003600E4F52822A3
:0237B3008F5A2B
:1037B500900118E0FFE55A7006E545D39F5012E5E4
:1037C5005A640160030238A9E546D39F50030238C5
:1037D500A9E55A7018C3E5459FF55D74602FF5821C
:1037E500E4341EAD82F55E8D5F7F40801BE55AB4E3
:1037F5000119C3E5469FF55D74B02FF582E4341ECB
:10380500AF82F55E8F5F7F101200167FF47E011286
:103815006D667D207F051267D07D1A7F081267D0FF
:103825007FC87E00126D66E4F55BE55BC3955D5070
:1038350061055FE55FAE5E7002055E14F5828E83FD
:10384500E0F55C123A5E38860038640A38680B3851
:103855006E0C38740D387A0E38800F0000388CE401
:10386500FD80277D5F7F0780227D5E7F06801C7D32
:103875000A7F0280167D327F0280107D467F02809E
:103885000A7D0A7F038004AD5CE4FF1267D0055B07
:103895008098E55A70047F408007E55AB401057F9A
:0438A50010126FC1CD
:0138A90022FC
:10517A00200E10754406901DB8E06003D20E22E49A
:10518A00F54222E528D394004003152822C2CA1505
:10519A0044E54414603D14603214601D1460151413
:1051AA007049901DB8E0FF7003F54222122C44901A
:1051BA001DB9802F901DBA8015901DBBE0FF7003AA
:1051CA00F54222122C44901DBC8018901DBDE0FFB0
:1051DA00020026901DBEE0FF7003F54222122C4405
:1051EA00901DBFE0FF120026D2CA22E4F542C2CACD
:0351FA00C20E22C0
:10674B00900028E0FF6026200E07124EB975281422
:10675B0022E528D394004003152822202708D2CA0B
:0E676B00752814D22722C2CA75287DC22722A3
:1066ED00200E0C7F1C124EB975286475783C22E57E
:1066FD0028D394004003152822AF781578D3EF6482
:0E670D00809480400475286422C20EE4F54298
:01671B00225B
:1063F200E54214601C14601C14601F1460221460B7
:106402002224057021C2CAC20EC227C21DE4F5446D
:106412002202517A12674BD21E22124239D21E2216
:076422000266ED1252FB229D
:10650000BF010790002A7418F022BF020790002AEA
:106510007412F022BF030590002A8014BF04079074
:10652000002A740BF02290002ABF05047409F0229F
:04653000740CF022D5
:0250F400AC0707
:1050F600C3EC64809480404AEC64809488504320DA
:105106002B21E4FD124EC3C333CE33CED8F9124E53
:105116003E74102BF58274003AF583EFF00DBD084E
:10512600E3801FE4FD124EC3C333CE33CED8F9124B
:105136004E3E74182BF58274003AF583EFF00DBDE0
:1051460008E3202B16E4FDEDFF3395E0FE74102FE7
:10515600F5827400124E6FBD08ED22302B15E4FD6A
:10516600EDFF3395E0FE74182FF5827400124E6F32
:03517600BD08ED84
:015179002213
:10506D007D3F7F091267D07D507F081267D0907009
:10507D003E1250EB7D5B7F061267D090703F125051
:10508D00EB907040E493FDE4FF1267D0907041E423
:10509D0093123A5E50BD4150C14250C54350CB446E
:1050AD0050D14550D74650DD4750E348000050EAF7
:1050BD007D0A80067D3280027D467F02801C7D0A3E
:1050CD007F0380167D287F0380107D467F03800A35
:1050DD007D0A7F0480047D287F041267D022E4932B
:0750ED00FDE4FF1267D02271
:106077008F5BE55B7005D22DFF8009E55BB40107F7
:10608700D22D7F01125B117D4B7F021267D07D02FB
:10609700E4FF1267D07D32E4FF1267D012506DE53E
:1060A7005B70028005E55BB401057F40126FC1227A
:103E1500A209300501B350307D017F04124FE550F2
:103E25002320050E30090B9000A4E0FF7C0B7D607C
:103E3500800F30050F20090C9000A5E0FF7C0B7D5D
:103E450080125CE4A2099205A20A300601B3503043
:103E55007D027F04124FE5502320060E300A0B9099
:103E650000A6E0FF7C0B7DA0800F30060F200A0C1A
:103E75009000A7E0FF7C0B7DC0125CE4A20A9206CD
:103E8500A20B300701B350307D037F04124FE5507C
:103E95002320070E300B0B9000A8E0FF7C0B7DE084
:103EA500800F30070F200B0C9000A9E0FF7C0C7DE4
:103EB50000125CE4A20B9207A20D300801B350304A
:103EC5007D047F04124FE5502320080E300D0B9022
:103ED50000AAE0FF7C0C7D20800F30080F200D0C20
:103EE5009000ABE0FF7C0C7D40125CE4A20D9208D3
:013EF50022AA
:10662D00534103900024E0FE543FFF78040880019D
:10663D0023D8FD54F0FFEE30E4034307049000240B
:0F664D00E030E503430708EF4241C2AF124E6051
:01665C00221B
:022992008F6B49
:10299400302F05756CF48003756C64E56B6401700D
:1029A40029AF417803EF08800123D8FD3392307FAB
:1029B4001020300B122AAE7F10127002022AA612C7
:1029C4002AB97F10127015022AA6E56B64027028DA
:1029D400AF417802EF08800123D8FD3392307F2085
:1029E40020300A122AAE7F201270028008122AB9FF
:1029F4007F20127015022AA6E56B64037028AF418C
:102A04007801EF08800123D8FD3392307F402030D5
:102A14000A122AC47F401270028008122ACF7F4013
:102A2400127015022AA6E56B6404701EE541339208
:102A3400307F8020300A122AC47F801270028008FE
:102A4400122ACF7F801270158058E56B64057027B9
:102A5400AF417805EF08800123D8FD3392307F041D
:102A640020300A122ADA7F041270028008122AE542
:102A74007F04127015802BE56B6406702CAF4178CF
:102A840004EF08800123D8FD3392307F0820300AF8
:102A9400122ADA7F081270028008122AE57F0812CF
:092AA4007015AF6C7E00126D6626
:102AAD0022127015AF6C7E00126D6622127002AF8D
:102ABD006C7E00126D6622127015AF6C7E00126D69
:102ACD006622127002AF6C7E00126D6622127015B6
:102ADD00AF6C7E00126D6622127002AF6C7E00121A
:032AED006D6622F1
:105E5700900024E030E0057F10127015900024E0D8
:105E670030E1057F20127015900024E030E2057FB5
:105E770040127015900024E030E3057F8012701502
:105E8700900024E030E4057F04127015900024E0B0
:095E970030E5057F0812701522A8
:106DB70030030A124EA4C203C211C21E22300409B4
:0A6DC700124EA4C204C213C21E2221
:10665D008F708D71E570B4011FE5717003125D7A55
:10666D00E571B40107787FE6FF125BB4E571B432D2
:10667D000E7FF47E01026D66AD71AF701267D02290
:1067D000EFFEEDFF1280008E2D8F2E1254E17574A6
:1067E00032AF741574EFD39400400EE4F573E57383
:0967F000C3943A50EC057380F5E6
:0167F900227D
:1054E100D2A8AFA875A881C214852E82852D83E428
:1054F10093C4540FFE4306F08E80C284D28500C24D
:10550100870000D287007580FF7580FEC284C28546
:1055110000C2870000D287007580FFD2147D407CD5
:105521001FE4FE30B40D0EBE32F9ED1D70011CED0D
:105531004C70EE7C1F7D40E4FE20B40D0EBE32F9AE
:10554100ED1D70011CED4C70EE8FA8C2A87F0A7E84
:0455510000126D6671
:015555002233
:1067FA007580FDC284C28500C28700000000D2876E
:10680A00007580FF7F0A7E00126D667F997E0912ED
:0A681A0080008E2D8F2E1254E12213
:1042FA00D284D285C286A2809217A2819220A282FB
:10430A009218A2839221D2862001537D027F011244
:10431A004FE540137D037F01124FE5400A3017072E
:10432A00301932D22480377D027F01124FE5500FB7
:10433A0030170C302009301904D224802180167DD0
:10434A00037F01124FE5501220170330200C301959
:10435A0004D224800912689E8004C219C224200251
:10436A004E7D027F02124FE540127D037F02124FFB
:10437A00E54009301806301B2FD225227D027F0224
:10438A00124FE5500E30180B302108301B03D2258E
:10439A002280157D037F02124FE5500F201803304B
:1043AA002109301B03D225220268C6C21BC225225C
:10689E00753D1E753E60E4FFE53E2FF582E4353D05
:1068AE00F583E4F00FBF50F0753D1E753E60E4F5C4
:0768BE0045C226C211D219E8
:0168C50022B0
:1068C600753F1E7540B0E4FFE5402FF582E4353F85
:1068D600F583E4F00FBF10F0753F1E7540B0E4F588
:0768E60046C228C213D21BB9
:0168ED002288
:106CF400C284D285C286A2809209A281920AA2820B
:0D6D0400920BA283920DD286D284D28522FA
:10622800E57D2560F582E4357CF5832274FF123A1A
:1062380034E4FBFAF9F8C3023A21057E7480257D1F
:10624800F57DE4357CF57C22F582E4341DF5832266
:0B625800757E01757C00757D20E4223E
:1043BA007D027F07124FE550057F04127002C22961
:1043CA00D223E4F5427FE87E03126D66C298C2AF3B
:1043DA00C2307F03122ECA755E7F755D96755C9832
:1043EA00755B00785B126234504430983E120006C6
:1043FA00126F18EF14601824F0602624C1600B2491
:10440A00F670287F061270278021126312801C7FA3
:10441A0006127027126AD212662D125EE8D229801D
:10442A000A7F06127027125B64D2293029B5E47814
:10443A0084F6D2307F01122ECA7F40120016C22F94
:10444A00126A8C7D467F021267D07D1E7F07126733
:10445A00D07D147F081267D07D327F031267D0C2E5
:0D446A00307F03122ECA7FFF126FC1C223E4
:014477002222
:105B6400126258F55F7F02127027E57E2402F56108
:105B7400AF7E127027E4F560126228E0FF127027EE
:105B8400126228E02561F5610560E560C3948040F8
:105B9400E7AF611270277F0312702712702FEF6432
:0F5BA40015600C126242055FE55FC3942240B6A4
:015BB30022CF
:106AD200126258F55F12653450077F0612702780E4
:106AE200057F15027027126242055FE55FC394229B
:026AF20040E37F
:016AF400227F
:10653400E4F56012702F74D02560126250EFF005FC
:1065440060E560C3948440EB126EF6901E52E0B591
:106554000710AE7CAF7DBE0504BF200100126D4A5A
:03656400D322C37C
:016567002211
:106D4A00E4FF74D22FF582E4341DF583E0FEE57D7D
:0B6D5A002F12622CEEF0000FBF80E74C
:016D6500220B
:106EF600E4FFFE74D02E126250E02FFF0EBE82F326
:016F06002268
:10631200E4F55FF5657564E0756393756204F56194
:10632200786112623450213098F61200068F60E5CF
:106332006064046013AF65056574D02F126250E586
:0863420060F0255FF55F80D8D3
:01634A002230
:04000600AF99C29854
:01000A0022D3
:087027003099FDC2998F9922F6
:07702F003098FDAF99C298F3
:017036002237
:106E04000C0102030405060708090A0B0C0102031E
:086E14000405060708090A0B3A
:10684D00AF5FEF3395E0FE75F007EF123A52EE753C
:10685D00F007A42583F583E0227882E6FF126DEB25
:09686D00EF22C295D297D2AF22AE
:10698A00C22CC2AF1270377F83126E1C126C0312B4
:10699A00686F7883E66F600B125FB3302B05126065
:0569AA00B7922CA22CA5
:0169AF0022C5
:1060B7007983E778866660367883E6FF7886F6EF39
:1060C7007013E552C3940A500C7D077F04124FE505
:1060D7005003125F2D7D057F04124FE55010E541F7
:1060E70054036005123FD6D322123FD6C322C322E0
:103FD600E4F55F900A5012684D700302409A900A09
:103FE600511268546016788066600302409A900AFF
:103FF6005212684D788766600302409AAF5FEF33CE
:1040060095E0FE900A53126854FF787FE6FEEF6E45
:104016006020EF601DB4080BEED394014005EE94CA
:1040260007400FEF6409706CEE64016005EE6407EB
:104036007062AF5FEF3395E0FE900A54126854FF4A
:10404600F46006EF788266704BE55FFD3395E0FC21
:10405600900A5575F007ED123A52EC12685C7883B7
:10406600667031D201D20274BD2DF58274003CF522
:1040760083E0FFC007EDAE047805C333CE33CED858
:10408600F92480F582740E3EAD82FCD007125CE402
:10409600C201C202055FC3E55F64809493500302C8
:0240A6003FD900
:0140A80022F5
:105F2D007D087F04124FE5500D7882E6FF126DEB70
:105F3D00EFC39407402CD2307F01122ECA7F40123E
:105F4D000016C22F126A8CD201D202E4FD7F0A1212
:105F5D004A13C201C2027F50126FC1C2307F0112BB
:035F6D002ECA2217
:105FB300C2AF1270377FBF126E1C126C037883A6B8
:105FC30007126C037883A607126C037882A6071264
:105FD3006C037887A607126C037880A607126C03FC
:105FE300787FA607126C037881A6071270371268B0
:025FF3006F221B
:105A0800C2AF1270377F8E125A577F90126E1C7F6A
:105A1800A7126E1C1270377FBE126E1CE4FF126E46
:105A28001C7883E6FF126E1C7882E6FF126E1C78E3
:105A380087E6FF126E1C7880E6FF126E1C787FE600
:105A4800FF126E1C7881E6FF125A5712686F2212F5
:0B5A58006E1CE4FF126E1C127037225F
:105BB4008F72E572B401047D63803EE572B402061F
:105BC4007D087F068035E572B403067D317F088049
:105BD4002AE572B404067D617F08801FE572B4056E
:105BE400067D257F088014E572B406067D597F037F
:0F5BF4008009E572B407077D487F071267D0224A
:026DEB00AE07F1
:106DED00EE54F0FF780408800103D8FD75F00AA475
:066DFD00FFEE540F2FFF12
:016E0300226C
:105D7A00126866906E0493FF1235B87883126868C9
:105D8A00601B7883126868C3940A50077D327F06C5
:105D9A001267D07883E6FF126DEB1235B812686687
:105DAA00C3940C50067D0A7F0280047D507F061240
:0A5DBA0067D07D507F051267D022EC
:105ABB007FF47E01126D667D097F061267D07880B8
:105ACB00125B017D0E7F031267D07D357F06126757
:105ADB00D07D097F061267D07887125B017D1E7F10
:105AEB00091267D07D1E7F071267D07881E6FF12FF
:105AFB006DEB1235B822E6FF126DEB1235B87FF461
:065B0B007E01126D66220E
:07703700C2B6C295D29522FA
:106E1C00E4FEC297EF30E002D297C2B6D2B6EFC30F
:066E2C0013FF0EBE08EC8E
:016E3200223D
:106C0300E4FFD297FED2B6C2B6A297E433C43333BD
:0F6C1300335480FDEFC313FFED42070EBE08E6BA
:016C2200224F
:10595000EF3395E0FE74702FF58274003EF583E01E
:10596000FF22AF5AEF3395E0FEEF222460F58274F8
:10597000013EAD82FCD22922900520E0F547A3E04C
:10598000F548222450F58274053EAD82FC22900039
:10599000BAE0FF7C0E7D2022D222D201E4FF22C297
:0D59A00001C2227F1922D222D2307F0222C2
:10283100E5527008126FEB8F5202292CE552B40554
:10284100081245EA8F5202292CE552B40B08126D89
:10285100818F5202292CE552B40A08125DC48F52AD
:1028610002292CE552B40F08125F708F5202292CF5
:10287100E552B414081223408F5202292CE552B4B8
:102881001908126C608F5202292CE552B41E0812ED
:102891006B3B8F5202292CE552B42308126BA18F96
:1028A1005202292CE552B42807126FCF8F52807B38
:1028B100E552B42D071269168F52806FE552B4327A
:1028C1000712634B8F528063E552B43E07126C7E50
:1028D1008F528057E552B43C07126EC08F52804B25
:1028E100E552B43307126B7F8F52803FE552B441FA
:1028F10007126F498F528033E552B44C07126F595A
:102901008F528027E552B44407126F698F52801BA2
:10291100E552B437071257D88F52800FE552B439B8
:10292100071255568F528003E4F552E55370061293
:10293100000E8F5322E553B4050612701E8F5322E9
:10294100E553B40A06126F798F5322E553B40F068B
:10295100126F888F5322E553B41406123C518F53E2
:1029610022E553B43D06126C9C8F5322E553B43FCC
:102971000612668D8F5322E553B443061268EE8F1B
:102981005322E553B44D06126BC28F5322E4F55323
:012991002223
:0D6FEB0090052AE0F52BA3E0F52C7F052290
:1045EA00302414201011C21C7D047F01124FE550A3
:1045FA00037F0B227F0A227F081264295006124782
:10460A00557F0022202408301005C2107F05227D24
:10461A00057F06124FE5501EE5394538701890009F
:10462A00B5E0FF7C0D7D80125CE490052EE0F53844
:10463A00A3E0F53980517D067F06124FE5501EE54D
:10464A003C453B70189000B6E0FF7C0D7DA0125CE3
:10465A00E4900530E0F53BA3E0F53C802A7D077F36
:10466A0005124FE5500B300008E52C452B7002C2AD
:10467A0000300F08E52C452B7002C20F7884E6B48F
:10468A0005057F04125379E551700875510AD22B3A
:06469A0012698A7F05226F
:106D8100200F1590053BE0F54E2024037F0522E5F9
:0B6D91004ED3940050F3D20F7F0A2273
:105DC4007D077F05124FE5500C7D077F05124FE5D7
:105DD400503230002F7D017F01124FE55026D23022
:105DE4007F01122ECA7F011200167D027F07124F17
:105DF400E550057F041270159000A0E0FF7C0A7D39
:0A5E0400E0125CE41259787F0F22CF
:105F700030243DE5484547700C7D087F01124FE510
:105F800050037F372230030EE53A700A126DB77F57
:105F90000112001680173026037F14227884E6B49D
:105FA000050B7F031253792024037F14227F0F22D5
:035FB0007F142239
:1023400090053DE0F54B7F01126FC1126DB77D0224
:102350007F07124FE55009E54B70057F04127002AC
:102360009000A1E0FF7C0B7D00125CE4D22B12698F
:102370008AE545700302246A7C017D001224F25034
:10238000037F3E227C017D501224D250037F3C22E9
:102390007C017D581224D250037F3C227C017D10A9
:1023A0001224DA50081224E250037F33227C017D8C
:1023B000201224DA500B9000BBE0FF7C0E7D4080A1
:1023C000207C017D281224EA500512598E80127C4F
:1023D000017D301224EA50129000B9E0FF7C0E7D9E
:1023E00000125CE412689E7F00227C017D40D229AD
:1023F000E4FF12496A500C7D067F04124FE550033A
:102400007F4C227C017D381224F250037F44227CD1
:10241000017D18C229E4FF12496A500C7D057F0135
:10242000124FE550037F4122E4F55A1259627803B6
:10243000C333CE33CED8F912596BE4FF12496A5038
:102440001BAF5A125950C0071259627805C333CED8
:1024500033CED8F9125983D007125C99055AC3E5D7
:102460005A648094A840C47F19221224E2500C7D43
:10247000077F05124FE5504B3000487884E6700422
:102480007F0180087884E6B404077F0212537980C4
:102490002F7884E6B40704760180257D037F061239
:1024A0004FE5501CE557455670169000AFE0FF7C95
:1024B0000C7DC0125CE4900532E0F556A3E0F557C0
:1024C0007F19227D077F05124FE550052000027F0E
:0124D0000506
:1024D10022D229E4FF12496A22D229E4FF12496A71
:1024E100227D077F05124FE522D229E4FF12496AB6
:0924F10022C229E4FF12496A220B
:106C600030260312689E7D077F05124FE5500620EF
:0E6C700000037F0522900538E0F54E7F1E22BE
:106B3B00E54E70037F23227D027F07124FE550093C
:106B4B00E54B70057F041270023024037F0A227F0D
:026B5B001E22F8
:106BA1001259787D067F01124FE5500C9000ACE040
:106BB100FF7C0C7D60125CE4900539E0F54E7F2D81
:016BC10022B1
:0E6FCF007FA0126FC1900539E0F54E7F2D2294
:10691600D22B12698A7D027F07124FE55009E54B9B
:1069260070057F04127002E54E70037F3222302418
:07693600037F0A227F2D22DE
:10634B00301E037F32227D047F06124FE5501FE57E
:10635B0055455470199000B0E0FF7C0C7DE0125C49
:10636B00E4900534E0F554A3E0F5557F3222C230BA
:08637B007F01122ECA7F0022EF
:106EC00020220CD222E4FF12055BC2227F00227F27
:026ED0003C2262
:106C7E00202218D2227F40120016D201121D87C286
:0E6C8E00017F40126FC1C2227F19227F3E2279
:106F490020220A1259981237B312599F227F4122DF
:106F590020220A1259981261EC12599F227F442269
:106F690020220A1259981255C612599F227F44228B
:05000E0000007F052247
:09701E003025037F0A227F0522C0
:0F6F79009000A2E0FF7C0B7D20125CE47F0F22D2
:0F6F88003025093028037F14227F0F227F142227
:103C51009000A3E0FF7C0B7D40125CE4E54670031D
:103C6100023D297D017F03124FE550707C017D08E3
:103C7100C2297F0112496A50037F3F227C017D5096
:103C8100123D2C50037F3D227C017D58123D2C506A
:103C9100037F3D227C017D40D2297F0112496A5078
:103CA1000C7D067F04124FE550037F4D227C017D80
:103CB10028D2297F0112496A500912598E125CE4F7
:103CC1007F00227C017D18C2297F0112496A500CB4
:103CD1007D057F02124FE550037F43227D027F0362
:103CE100124FE55043E4F55AAF5A1259647803C3B1
:103CF10033CE33CED8F912596B7F0112496A501D68
:103D0100AF5A125950C007AF5A1259647805C333DC
:103D1100CE33CED8F9125983D007125C99055AC314
:0A3D2100E55A648094A840C07F00BA
:093D2B0022D2297F0112496A220B
:106C9C00202218D222C2307F01122ECA7F01126F1D
:0E6CAC00C17F0112055BC2227F00227F3D22C4
:10668D0020222A1259A6122ECA7FF47E01126D669F
:10669D007F10120016D202121B86C2027F10126FDB
:1066AD00C1C2307F02122ECAC2227F00227F3F223A
:1068EE002022221259A6122ECA7FF47E01126D6644
:1068FE00D2027F011237B3C202C2307F02122ECAF9
:08690E00C2227F00227F432218
:106BC20020221B1259A6122ECAD2027F011261EC98
:106BD200C202C2307F02122ECAC2227F00227F4D21
:016BE2002290
:10563400AF5AEF3395E0FE22900520E0F547A3E052
:10564400F54822900522E0F549A3E0F54A222460BA
:10565400F58274013EAD82FCD2292274702FF5824A
:1056640074003EF583E0FF22C202C2227F19222485
:1056740050F58274053EAD82FC22900536E0F53289
:10568400A3E0F53322055AC3E55A648094A822D2D4
:0D56940022C2307F0122D222C2307F0222CA
:10326500E5527006126B5D8F5222E552B4050612C7
:1032750036B78F5222E552B40B0612693D8F5222A2
:10328500E552B40A061244788F5222E552B40F066D
:10329500126ED28F5222E552B411061258958F52F2
:1032A50022E552B412061251FD8F5222E552B41492
:1032B50006120A548F5222E552B4190612671C8F62
:1032C5005222E552B41E061266BD8F5222E552B453
:1032D50023061260368F5222E552B42806126FDD9E
:1032E5008F5222E552B42D061262638F5222E552A7
:1032F500B432061263838F5222E552B43C06126E35
:10330500E48F5222E552B43D06126D9C8F5222E5A0
:1033150052B43E06126A1F8F5222E552B43F06127E
:103325006F078F5222E552B44106126C238F522249
:10333500E552B44306126AF58F5222E552B44C06A3
:10334500126DD18F5222E552B44D06126B188F5271
:1033550022E552B437061257D88F5222E552B439B6
:10336500061255568F5222E552B438061267A58FBC
:103375005222E552B43306126B7F8F5222E552B4C6
:0C3385004406126E338F5222E4F55222EF
:106B5D0090052AE0F52BA3E0F52C7D067F02124F60
:106B6D00E5500C90052CE0F529A3E0F52AD21F7F06
:026B7D000522EF
:1036B700302414201011C21C7D047F01124FE550E5
:1036C700037F0B227F0A22302514201211D21C7D82
:1036D700047F02124FE550037F0B227F0A227F08E7
:1036E70012642950061247557F0022202408301003
:1036F70005C2107F0522202508301205C2127F055A
:10370700227D057F06124FE5501EE53945387018B2
:103717009000B5E0FF7C0D7D80125CE490052EE003
:10372700F538A3E0F53980757D067F06124FE55021
:103737001EE53C453B70189000B6E0FF7C0D7DA070
:10374700125CE4900530E0F53BA3E0F53C804E7D4C
:10375700077F05124FE5500D30000AE52C452B7009
:1037670004C200800B300F08E52C452B7002C20FF6
:103777007D067F02124FE55019301F16E52A4529AD
:103787007010C21F9000BCE0FF7C0E7D60125CE4ED
:10379700800B7884E6B405057F04125379E55170F0
:0C37A7000875510AD22B12698A7F052296
:10693D00200F2190053BE0F54E202406201C037FFF
:10694D000522202506301C037F0522E54ED3940039
:07695D0050E7D20F7F0A2270
:104478007D077F05124FE550127D077F05124FE536
:104488004003024529200003024529201C3FD23061
:104498007F03122ECA7F0F126FC190000FE0B40283
:1044A800047F05800990000FE0B403057F01120026
:1044B8001612563C7D027F07124FE550057F041205
:1044C80070159000A0E0FF7C0A7DE0804E301C5102
:1044D80090000FE0FF64026005EF640370437F0FF4
:1044E800126FC17F05126429400BD2307F01122E52
:1044F800CA7F028009D2307F03122ECA7F0A1200B7
:10450800167D027F07124FE550057F0412701512C1
:1045180056479000A2E0FF7C0B7D20125CE47F0FE1
:0A4528002212563C1256477F0F2264
:106ED200201C063024037F1122301C053025027F3E
:026EE20012227A
:10589500302458E5484547700C7D087F01124FE5D7
:1058A50050037F3722300329E53A70257FA0126F18
:1058B500C190000FE0B401047F01800990000FE062
:1058C500B402057F05120016E4F542C21EC203802C
:1058D500173026037F14227884E6B4050B7F031264
:0E58E50053792024037F14227F11227F142286
:1051FD00301C1030240D20100A7F0A126FC1C21C02
:10520D007F0A22301C5230254F20124C30030312DE
:10521D006DB7E54A4549700C7D087F02124FE55088
:10522D00037F3822300417E53A70137FA0126FC147
:10523D007F02120016E4F542C21EC2048017302808
:10524D00037F14227884E6B4050B7F031253792073
:10525D0025037F14227F1222201C1230250F2012CD
:10526D000CD21CC2307F02122ECA7F0A227F14225A
:100A540090053DE0F54B7F0F126FC1201C0C9000F8
:100A6400A1E0FF7C0B7D00125CE4301C0C9000A321
:100A7400E0FF7C0B7D40125CE4E542B403037F1489
:100A840022126DB7E4F5427D027F07124FE550094B
:100A9400E54B70057F04127002D22B12698A301C58
:100AA40003020B97E5457003020B977C017D00124E
:100AB4000D1E50037F3E227C017D50120CEE50032C
:100AC4007F3C227C017D58120CEE50037F3C227C3B
:100AD400017D10120CF65008120D0650037F3322CC
:100AE4007C017D20120CF65003020BFE7C017D2854
:100AF400120D0E500C9000BAE0FF7C0E7D20020C0B
:100B0400077C017D30120D0E500C9000B9E0FF7C83
:100B14000E7D00020C077C017D40D229E4FF1249BE
:100B24006A500C7D067F04124FE550037F4C227CF3
:100B3400017D38120D1E50037F44227C017D18C2B2
:100B440029E4FF12496A500C7D057F01124FE550DC
:100B5400037F4122E4F55A125634EF7803C333CEAF
:100B640033CED8F9125652E4FF12496A501D125678
:100B74003412565FC007125634EF7805C333CE33B0
:100B8400CED8F9125673D007125C9912568940C711
:100B94007F1922201C03020C8AE5467003020C8A8A
:100BA4007D017F03124FE54003020C427C017D0866
:100BB400C2297F0112496A500F7F50120016D230A9
:100BC4007F02122ECA7F3F227C017D50120CFE5000
:100BD400037F3D227C017D58120CFE50037F3D2291
:100BE4007C017D10120D165008120D0650037F3340
:100BF400227C017D20120D1650129000BBE0FF7C78
:100C04000E7D40125CE412689E7F00227C017D40D0
:100C1400D2297F0112496A500C7D067F04124FE5E8
:100C240050037F4D227C017D18C2297F0112496A3D
:100C3400500C7D057F02124FE550037F43227D0255
:100C44007F03124FE5503CE4F55A125634EF780313
:100C5400C333CE33CED8F91256527F0112496A50AB
:100C64001D12563412565FC007125634EF7805C36E
:100C740033CE33CED8F9125673D007125C9912567C
:100C84008940C77F1922120D265008120D26504B99
:100C94003000487884E670047F0180087884E6B4E4
:100CA40004077F02125379802F7884E6B407047610
:100CB4000180257D037F06124FE5501CE5574556FC
:100CC40070169000AFE0FF7C0C7DC0125CE49005D0
:100CD40032E0F556A3E0F5577F19227D077F051210
:090CE4004FE550052000027F05D8
:100CED0022D229E4FF12496A22D229E4FF12496A6D
:100CFD0022D2297F0112496A227D077F05124FE515
:100D0D0022D229E4FF12496A22D2297F0112496AAF
:100D1D0022C229E4FF12496A227D077F05124FE5A1
:010D2D0022A3
:10671C00C219C2307F02122ECA30260512689E8022
:10672C00063028031268C67D077F05124FE5500618
:0F673C002000037F0522900538E0F54E7F1E22D6
:1066BD00E54E70037F23227D027F07124FE55009BF
:1066CD00E54B70057F041270023024062010037F05
:1066DD000A22302508201205D21C7F0A227F1E2295
:10603600201C0512563C80031256477D067F01122E
:106046004FE55024E5427020201C0B9000ACE0FF89
:106056007C0C7D60800C301C0C9000ADE0FF7C0C4D
:106066007D80125CE47F2822900539E0F54E7F2D75
:016076002207
:0E6FDD007FA0126FC1900539E0F54E7F2D2286
:10626300D22B12698A7D027F07124FE55009E54B55
:1062730070057F04127002E54E601D302406201065
:10628300037F0A2290000FE0640160093025062095
:0B62930012037F05227F2D227F3222A4
:10638300301E037F32227D047F06124FE5501FE546
:1063930055455470199000B0E0FF7C0C7DE0125C11
:1063A300E4900534E0F554A3E0F5557F3222C23082
:0863B3007F01122ECA7F0022B7
:106EE40020220CD222E4FF12055BC2227F00227F03
:026EF4003C223E
:106A1F0020221FC2307F02122ECAD2227F401200C4
:106A2F0016D201121D87C2017F40126FC1C2227F91
:056A3F0019227F3E2238
:106F070020220BD222D202121B8612566C227F3FFE
:016F17002257
:106D9C00202215125693122ECA7F40126FC17F010A
:0B6DAC0012055BC2227F00227F3D2207
:106C230020221912569A122ECA7F10126FC1D20156
:0F6C3300E4FF1237B3C201C2227F19227F412230
:106AF50020221D125693122ECA7F40126FC1D2302A
:106B05007F02122ECAD2027F011237B312566C22AF
:036B15007F432299
:106DD10020221412569A122ECAD201E4FF1261EC3B
:0A6DE100C201C2227F19227F412265
:106B180020221D125693122ECA7F40126FC1D23006
:106B28007F02122ECAD2027F011261EC12566C2229
:036B38007F432276
:106E330020221112569A122ECAD202E4FF1255C60C
:076E430012566C227F44226D
:1057D800D2107D027F07124FE550057F0412700238
:1057E80090000FE0FF64016004EFB4030E7F011224
:1057F8006FC17F401258277F01801390000FE0B4DB
:10580800020F7F05126FC17F501258277F03127055
:10581800027F50126FC130150312567E7F39221253
:0F5828000016C22F126A8CE4FD7F07124A13226A
:1055560030241130150BE53345327005C231126A1D
:10556600447F3922E47884F6C21090000FE0FF648D
:10557600016005EF64037010D2307F01122ECA7FDE
:10558600401255B47F01801B90000FE06402701634
:10559600D2307F03122ECA7F05126FC17F5012557B
:1055A600B47F03122ECA7F50126FC17F00221200F1
:1055B60016C22F126A8CE4FD7F08124A13C23022EB
:1067A500D2127F0A126FC17F40120016D22F126AD1
:1067B5008CE4FD7F07124A137F031270027F50128B
:0B67C5006FC130150312567E7F0022CA
:106B7F0030000B9000B8E0FF7C0D7DE0800C200012
:106B8F000E9000B7E0FF7C0D7DC0125CE4B2007F79
:026B9F001922B9
:1061EC008F5AE55A24FF922F126A8CE55A70127F4F
:1061FC0040120016D201E4FD7F09124A13C201803D
:10620C0015E55AB401107F10120016D202E4FD7F7E
:0C621C0009124A13C2027F50126FC12207
:10417300C201C202D20C7F50126FC17F801200169F
:1041830075420390000FE0640170323024297F01EF
:104193001200167D027F07124FE550057F0412704F
:1041A30015302404E54270F920240C7F0112422EBD
:1041B30050057F04127002E54270D0806490000FB6
:1041C300E0FF64026005EF640370563024357F021C
:1041D300126FC17F051200167F021270157D027FD8
:1041E30007124FE550057F04127015302404E54291
:1041F30070F92024287F0512422E50217F0412706B
:1042030002801A3025177F0212001620240730255A
:1042130004E54270F62025057F02126FC1E5427066
:10422300AA7FA0126FC1C20CC21E22126FC17D02EF
:064233007F07124FE52297
:03000000026D117D
:106D1100758E0078FEE4F6D8FD9000007FFF7E1F9F
:0D6D2100E4F0A3DFFCDEFA758187024DAEC1
:10399800C2D530F707B2D563F0FF05F030E70CB2B7
:1039A800D5F4048463F0FF05F080018430D502F477
:0239B8000422E7
:1039BA00EF8DF0A4A8F0CF8CF0A428CE8DF0A42E21
:0239CA00FE22DB
:1039CC00BC000BBE0029EF8DF084FFADF022E4CCDF
:1039DC00F875F008EF2FFFEE33FEEC33FCEE9DECA8
:1039EC00984005FCEE9DFE0FD5F0E9E4CEFD22EDEE
:1039FC00F8F5F0EE8420D21CFEADF075F008EF2F38
:103A0C00FFED33FD4007985006D5F0F222C398FD28
:053A1C000FD5F0EA22C5
:103A2100EB9FF5F0EA9E42F0E99D42F0E89C45F0FB
:013A31002272
:103A32007401FF3395E0FEFDFC080808E6CF2FF67F
:103A420018E6CE3EF618E6CD3DF618E6CC3CF62258
:0C3A5200A42582F582E5F03583F583227F
:103A5E00D083D082F8E4937012740193700DA3A3F7
:103A6E0093F8740193F5828883E47374029368600B
:063A7E00EFA3A3A380DF0B
:106F1800EFC39461400AEF947B5005EF24E0FF2211
:016F28002246
:00000001FF
